:0200000480007A
:10000000B72F0000938F0F8073900F306F00400365
:100010001300000013000000130000001300000094
:100020001300000013000000130000001300000084
:100030001300000013000000130000001300000074
:100040009702000093824211739052309300000097
:10005000130100009301000013020000930200004E
:100060001303000093030000130400009304000036
:10007000130500009305000013060000930600001E
:100080001307000093070000130800009308000006
:100090001309000093090000130A0000930A0000EE
:1000A000130B0000930B0000130C0000930C0000D6
:1000B000130D0000930D0000130E0000930E0000BE
:1000C000130F0000930F000097110200938181C469
:1000D00017050200130505479795030093854566AC
:1000E00013060000EF00001A170502001305053A79
:1000F000970502009385A54113060000EF008018C4
:1001000017A503001305056497B5030093854563A0
:1001100037B6ABAB1306B6BAEF00C01617B1030083
:1001200013014162EF80405B9392120093D2120060
:100130009382D2FF638A02008322010013014100EF
:100140006F0000177300203083220100130141006B
:10015000730020301301C1FF23205100F32220340B
:10016000E3C402FC8322010013014100130141F8A2
:1001700023221100232421002326310023284100BB
:10018000232A5100232C6100232E71002320810299
:10019000232291022324A1022326B1022328C10293
:1001A000232AD102232CE102232EF1022320010570
:1001B0002322110523242105232631052328410567
:1001C000232A5105232C6105232E71052320810745
:1001D000232291072324A1072326B1072328C1073F
:1001E000232AD107232CE107232EF107732520347E
:1001F000F3251034130601006F000000731015344E
:1002000083204100032181008321C10003220101D9
:1002100083224101032381018323C10103240102BD
:1002200083244102032581028325C10203260103A1
:1002300083264103032781038327C1030328010485
:1002400083284104032981048329C104032A010569
:10025000832A4105032B8105832BC105032C01064D
:10026000832C4106032D8106832DC106032E010731
:10027000832E4107032F8107832FC1071301C10775
:10028000730020302320C5006376B50013054500B8
:100290006FF05FFF678000000000000000000000BA
:1002A000000000000000000000000000000000004E
:1002B000130101F8232011002322210023243100FF
:1002C0002326410023285100232A6100232C71009A
:1002D000232E8100232091022322A1022324B10294
:1002E0002326C1022328D102232AE102232CF10272
:1002F000232E010323201105232221052324310568
:100300002326410523285105232A6105232C710545
:10031000232E8105232091072322A1072324B1073F
:100320002326C1072328D107232AE107232CF1071D
:100330009702020083A2C21823A02200F3221034E5
:10034000232E5106EF00C03B170102000321411785
:10035000032101008322C10773901234B7220000E9
:100360009382028873A00230832001000322C1001F
:100370008322010103234101832381010324C1015D
:100380008324010203254102832581020326C10241
:100390008326010303274103832781030328C10325
:1003A000832801040329410483298104032AC10409
:1003B000832A0105032B4105832B8105032CC105ED
:1003C000832C0106032D4106832D8106032EC106D1
:1003D000832E0107032F4107832F81071301010893
:1003E00073002030970202009382C21523A01200EE
:1003F00023A2220023A4320023A6420023A85200F5
:1004000023AA620023AC720023AE820023A09202D2
:1004100023A2A20223A4B20223A6C20223A8D202CC
:1004200023AAE20223ACF20223AE020323A01205A8
:1004300023A2220523A4320523A6420523A85205A0
:1004400023AA620523AC720523AE820523A092077E
:1004500023A2A20723A4B20723A6C20723A8D20778
:1004600023AAE20723ACF207EF60D06B170102006A
:1004700003210105032101008322C1077390123477
:10048000B72200009382028873A00230832001000B
:100490000322C1008322010103234101832381013F
:1004A0000324C10183240102032541028325810223
:1004B0000326C10283260103032741038327810307
:1004C0000328C103832801040329410483298104EB
:1004D000032AC104832A0105032B4105832B8105CF
:1004E000032CC105832C0106032D4106832D8106B3
:1004F000032EC106832E0107032F4107832F810797
:1005000013010108730020309702020093828203D6
:1005100083A0020003A1420083A1820003A2C200C3
:1005200083A2020103A3420183A3820103A4C201A7
:1005300083A4020203A5420283A5820203A6C2028B
:1005400083A6020303A7420383A7820303A8C2036F
:1005500083A8020403A9420483A9820403AAC20453
:1005600083AA020503AB420583AB820503ACC20537
:1005700083AC020603AD420683AD820603AEC2061B
:1005800083AE020703AFC20983AF82076780000012
:1005900073700430130101F823201100232221007D
:1005A000232431002326410023285100232A6100FF
:1005B000232C7100232E8100232091022322A102EB
:1005C0002324B1022326C1022328D102232AE102D7
:1005D000232CF102232E01032320110523222105C0
:1005E000232431052326410523285105232A6105AB
:1005F000232C7105232E8105232091072322A10797
:100600002324B1072326C1072328D107232AE10782
:10061000232CF1079702020083A282EA23A0220082
:10062000232E1106EF30C06D17010200032141E9AE
:10063000032101008322C10773901234B722000006
:100640009382028873A00230832001000322C1003C
:100650008322010103234101832381010324C1017A
:100660008324010203254102832581020326C1025E
:100670008326010303274103832781030328C10342
:10068000832801040329410483298104032AC10426
:10069000832A0105032B4105832B8105032CC1050A
:1006A000832C0106032D4106832D8106032EC106EE
:1006B000832E0107032F4107832F810713010108B0
:1006C00073002030737004306F00000073104530E9
:1006D000678000007325403073F04330678000006E
:1006E00097070000938747FE232EB5FE2322C5FA05
:1006F000232635F82320F5F8130505F86780000058
:10070000130101FF23261100EF60103FEF20501767
:10071000631805008320C1001301010167800000F8
:100720008320C100130101016F30805D93078500B4
:100730001307F0FF2322F5002324E5002326F5000C
:100740002328F500232005006780000023280500EA
:10075000678000008327450023A2F50003A78700D8
:1007600023A4E50003A787002322B70023A4B70032
:1007700023A8A50083270500938717002320F500F1
:100780006780000003A605009307F0FF13078500AC
:100790006316F6006F008003138707008327470066
:1007A00083A60700E37AD6FE23A2F50023A4B700B0
:1007B00023A4E5002322B70023A8A5008327050072
:1007C000938717002320F5006780000003270501A9
:1007D000832747006FF05FFD0327450083268500D0
:1007E000832705012324D70003278500832645009E
:1007F0002322D70003A747006316A700032785001D
:1008000023A2E7002328050003A507001305F5FF31
:1008100023A0A70067800000032605049387050036
:10082000630406028325C50003274500B385C50080
:100830002326B50063E6E500832505002326B500E1
:10084000138507006F50900767800000130101FFB8
:100850002324810023261100130405002322910084
:10086000EF30507D83278404635AF00483274402C9
:1008700063860704930444026F0000028327840404
:100880009387F7FF2324F404832784046358F0023A
:10089000832744026384070213850400EF30902805
:1008A000E30E05FCEF305055832784049387F7FF50
:1008B0002324F40483278404E34CF0FC9307F0FF23
:1008C0002324F404EF30507AEF30D07683274404A9
:1008D000635AF00483270401638607049304040128
:1008E0006F000002832744049387F7FF2322F40458
:1008F000832744046358F0028327040163840702BA
:1009000013850400EF301022E30E05FCEF30D04ECB
:10091000832744049387F7FF2322F40483274404A6
:10092000E34CF0FC9307F0FF2322F404032481003E
:100930008320C10083244100130101016F30D07274
:1009400063000508130101FF232481002322910085
:10095000130405002326110093840500EF30906DE9
:10096000832604048327C40303270400232C0402E2
:10097000B387F6021306F0FF2322C4042324E40005
:100980002324C404B386D740B307F7003307D70046
:100990002322F4002326E400639804028327040141
:1009A000639E0702EF30506C8320C1000324810056
:1009B000832441001305100013010101678000002A
:1009C000737004306F00000013050401EFF01FD6B0
:1009D00013054402EFF09FD56FF0DFFC130504010F
:1009E000EF30501493071000E31EF5FAEFF05FBAF2
:1009F0006FF05FFB63160500737004306F0000003A
:100A0000130101FE232A910023282101232631010D
:100A1000232E1100232C8100930906001389050061
:100A200093040500638E05083305B50213055505CB
:100A3000EF50404813040500630C05089307450573
:100A40002320F500232E940223202405EF30905E0E
:100A5000832604048327C403032704001306F0FF3E
:100A6000B387F602232C04022322C4042324E400C7
:100A70002324C40413050401B386D740B307F70049
:100A80003307D7002322F4002326E400EFF01FCA27
:100A900013054402EFF09FC9EF30105D23083405C1
:100AA000130504008320C101032481018324410133
:100AB000032901018329C10013010102678000009D
:100AC00013054005EF50003F1304050063160500B1
:100AD000737004306F000000232084006FF09FF6D5
:100AE00063160500737004306F0000006376B50074
:100AF000737004306F000000130101FF2324810094
:100B0000130620001384050093050000232611001E
:100B1000EFF05FEE630C0500232C85028320C100FB
:100B20000324810013010101678000007370043009
:100B30006F000000130101FB23261104232481040C
:100B40002322910423202105232E3103232C41034A
:100B5000232A510323286103232671032326C1007E
:100B600063060528638C052693072000639CF60026
:100B70000327C503930710006306F7007370043062
:100B80006F0000001389060093840500130405001C
:100B9000EF30902A631A05008327C100638607009F
:100BA000737004306F000000EF30D04803278403D7
:100BB0008327C403130B0000930B20009309F0FF5D
:100BC000130A0401930A44026364F710630479234F
:100BD0008327C1006382073663160B00130581016A
:100BE000EF30100FEF305048EF20803BEF30904453
:100BF0008327440463943701232204048327840455
:100C00006394370123240404EF3010469305C10098
:100C100013058101EF30D00E63160530EF3090419F
:100C2000032784038327C4036304F710EF30D04302
:100C3000EF305040832784046346F0026F000003C6
:100C400013850A00EF30006E63040500EF30D01A00
:100C5000832784049387F7FF2324F40483278404E1
:100C60006356F00083274402E39C07FC23243405E9
:100C7000EF30903FEF30103C832744046346F0028E
:100C80006F00000313050A00EF30C069630405001C
:100C9000EF309016832744049387F7FF2322F40450
:100CA000832744046356F00083270401E39C07FC78
:100CB00023223405EF30503BEF200062130B10006D
:100CC000EF305037032784038327C403E370F7F022
:100CD0000326040463040612631A091E0325840014
:100CE00093850400EF50803D83278400832604040D
:100CF00003274400B387D7002324F40063E4E710FC
:100D00008327840383260400032744029387170064
:100D10002324D400232CF40263000710130544029B
:100D2000EF304060930710006318F50E6F00401419
:100D3000EF3090338325C10013050A00EF30803176
:100D4000EF30502F832784046346F0026F000003C6
:100D500013850A00EF30005D63040500EF30D00911
:100D6000832784049387F7FF2324F40483278404D0
:100D70006356F00083274402E39C07FC23243405D8
:100D8000EF30902EEF30102B832744046346F0029F
:100D90006F00000313050A00EF30C058630405001C
:100DA000EF309005832744049387F7FF2322F40450
:100DB000832744046356F00083270401E39C07FC67
:100DC00023223405EF30502AEF200051E31805EEBE
:100DD000EFF00FFC130B10006FF09FEE832705045C
:100DE000E38407D8737004306F0000007370043020
:100DF0006F00000003260404631006088327040024
:100E0000638607048327840303274402938717001C
:100E1000232CF402E31407F0EF3010251305100023
:100E20008320C10403248104832441040329010491
:100E30008329C103032A8103832A4103032B01036E
:100E4000832BC102130101056780000003254400C4
:100E5000EF30501183278403032744022322040028
:100E600093871700232CF402E31A07EAE30605FA36
:100E7000EFF00FF26FF05FFA0325C40093850400D2
:100E8000EF50C023832704040327C40083260400F3
:100E9000B307F0403307F7002326E400637ED7044E
:100EA00003274400B307F7002326F40013072000AC
:100EB000832744026304E90403278403130717000C
:100EC000232CE402E38A07F46FF05FE50325C400F6
:100ED00093850400EF50801E832704040327C40079
:100EE00083260400B307F0403307F7002326E4000D
:100EF000E37ED7FA6FF0DFFA8327440203278403E7
:100F0000E30C07FA032784031307F7FF232CE402FB
:100F10000327840313071700232CE402E38E07EE54
:100F20006FF0DFDF13050400EFF05F92EF20C03AAF
:100F3000130500006FF0DFEEEF3010131305000013
:100F40006FF01FEE130101FF2322910093040500AF
:100F5000130540052324810023261100EF409075DE
:100F600013040500630C0504232C05029307F0FF0E
:100F70002322F5041307100013050501232EE402B4
:100F80002324F40423220400232004002324040047
:100F9000232604002320040423089404EFF00FF90F
:100FA00013054402EFF08FF89306000013060000CB
:100FB0009305000013050400EFF0DFB713050400EC
:100FC0008320C10003248100832441001301010117
:100FD0006780000063040504130101FF23248100DE
:100FE00023229100232611002320210103294500FB
:100FF00013040500EF304063930400006304A9026A
:101000008320C1000324810013850400032901000B
:1010100083244100130101016780000073700430D4
:101020006F0000008327C400930410009387F7FF2C
:101030002326F400E39607FC930600001306000045
:101040009305000013050400EFF0DFAE6FF05FFBC7
:10105000130101FC232E1102232C8102232A910269
:101060002328210323263103232441032326C100FF
:10107000630E050A930900006384051013890600B6
:101080009384050013040500130A05016F00800313
:10109000EF30807DEF30007A9305C10013058101A8
:1010A000EF30004663100506EF30C0780327840355
:1010B0008327C403630CF702EF30007BEF30C07A64
:1010C00093091000EF300077032784038327C403BC
:1010D0006362F7068327C10063860702E39A09FA71
:1010E00013058101EF30C03E6FF09FFAEF30C077FB
:1010F0008325C10013050A00EF20D075EFF04FC91A
:101100006FF0DFFBEF3040768320C10303248103BF
:1011100083244103032901038329C102032A810295
:101120001305000013010104678000007370043090
:101130006F000000032604046314060683270400DE
:1011400063880704832784030327440293871700D7
:10115000232CF40263100708EF3000718320C103D1
:101160000324810383244103032901038329C1024A
:10117000032A810213051000130101046780000097
:1011800083270504E38C07EE737004306F000000C2
:1011900003254400EF30005D232204006FF09FFA26
:1011A000631609040325840093850400EF40107141
:1011B000832784008326040403274400B387D700D1
:1011C0002324F400E3E0E7F8832704002324F40059
:1011D0006FF05FF713054402EF30C014930710005F
:1011E000E31CF5F6EFF0CFBA6FF01FF70325C4004C
:1011F00093850400EF40906C832704040327C40008
:1012000083260400B307F0403307F7002326E400E9
:101210006378D70003274400B307F7002326F400C0
:1012200093072000E310F9F283278403E38C07F08F
:10123000832784039387F7FF232CF4026FF09FF03A
:10124000130101FC232E1102232C8102232A910277
:101250002328210323263103232441032326C1000D
:101260006308051493040000638C0512938906003B
:101270001389050013040500130A45026F000001DD
:10128000EF30805EEF30405E93041000EF30805A04
:1012900083278403639E07088327C100638C0704A8
:1012A00063840404EF30405CEF30C0589305C10004
:1012B00013058101EF30C024631E0502EF30805713
:1012C00083278403E39E07FAEF30005A8327040044
:1012D000638607048325C10013050A00EF20905799
:1012E000EFF00FAB6FF01FFA13058101EF30401ED6
:1012F0006FF05FFBEF3040578320C103032481036D
:1013000083244103032901038329C102032A8102A3
:10131000130500001301010467800000EF308051C5
:1013200003254400EF300034EF3000546FF09FFA93
:10133000032604048324C400630406020327440034
:10134000B387C4002326F40063E6E7008327040084
:101350002326F4008325C40013050900EF4010562E
:10136000639C090483278403032704009387F7FF02
:10137000232CF40263160700EF3040562322A4000A
:10138000832704016380070413050401EF2090798B
:10139000930710006318F502EFF08F9F6F00800233
:1013A00083270504E38407EC737004306F000000AA
:1013B000737004306F0000008327440223269400DA
:1013C00063960702EF30404A8320C1030324810360
:1013D00083244103032901038329C102032A8102D3
:1013E0001305100013010104678000001305440277
:1013F000EF205073E30805FC6FF01FFA6302050A43
:1014000063880508130101FE232C8100232A910023
:101410002328210123244101232E110023263101F9
:10142000930720009384060013090600138A050021
:1014300013040500639CF6000327C50393071000FF
:101440006302F70A737004306F000000EFF08FA89A
:10145000032784038327C403930905006366F70405
:101460009304000013850900EFF04FA68320C1010B
:101470000324810113850400032901018324410110
:101480008329C100032A8100130101026780000043
:1014900083270504E38807F6737004306F000000AB
:1014A000737004306F00000003260404631E060CF2
:1014B0008327040063860712832784031307F0FF42
:1014C00093871700232CF402832784046388E70E94
:1014D0008327840493041000938717002324F404C3
:1014E0006FF05FF8EFF00F9F032784038327C40397
:1014F000930905006360F70603260404E30A06FA6D
:101500000325C40093050A00EF40503B83270404E1
:101510000327C40083260400B307F0403307F70015
:101520002326E4006378D70003274400B307F700BD
:101530002326F40093072000E390F4F88327840324
:10154000E38C07F6832784039387F7FF232CF402A9
:101550006FF09FF603260404E30C06F40325C40091
:1015600093050A00EF409035832704040327C40045
:1015700083260400B307F0403307F7002326E40076
:10158000E364D7FA6FF09FFBE39C04F60325840025
:1015900093050A00EF4090328327840083260404D9
:1015A00003274400B387D7002324F400E3E6E7F0E1
:1015B000832704002324F4006FF01FF083274402E4
:1015C00093041000E38007EA13054402EF209055CE
:1015D000E30A05E8E30809E8232099006FF09FE893
:1015E00003254400EF300018232204006FF0DFECE5
:1015F0006302050A832705046386070073700430BD
:101600006F00000083270500638A0708130101FEAD
:10161000232C8100232A9100130405002328210193
:1016200023263101232E110013890500EFF08F8A44
:10163000032784038327C403930905009304000050
:101640006376F702832784031307F0FF938717005D
:10165000232CF40283278404638AE7048327840409
:1016600093041000938717002324F40413850900C2
:10167000EFF0CF858320C10103248101138504008D
:1016800003290101832441018329C10013010102BF
:1016900067800000737004306F00000083274500EE
:1016A000E38607F6737004306F000000832744025E
:1016B00063960700930410006FF05FFB130544026C
:1016C000EF205046E30805FEE30609FE93071000ED
:1016D0002320F9006FF01FFE130101FC232E1102DD
:1016E000232C8102232A910223282103232631035C
:1016F00023244103232251032326C1006306052826
:10170000638C0526938A060093890500130405005F
:10171000EF209072631A05008327C10063860700DB
:10172000737004306F000000EF30C0108327840313
:101730006394071C8327C100638007101305810190
:10174000EF2010599304F0FF13094402130A040117
:10175000EF308011EF10D004EF30C00D8327440428
:1017600063949700232204048327840463949700DE
:1017700023240404EF30400F9305C10013058101B9
:10178000EF20105863100524EF30C00A832784032C
:10179000638A070AEF30400DEF30C00983278404C5
:1017A0006346F0026F00000313050900EF20903735
:1017B00063040500EF205064832784049387F7FFB8
:1017C0002324F404832784046356F000832744020F
:1017D000E39C07FC23249404EF300009EF308005DC
:1017E000832744046346F0026F00000313050A00D8
:1017F000EF20503363040500EF201060832744047A
:101800009387F7FF2322F404832744046356F000F0
:1018100083270401E39C07FC23229404EF30C004D7
:10182000EF10902BEF300001832784036396070CA1
:101830008327C100E39E07F0EF300003130500008B
:101840006F00800FEF304002832704006388071089
:101850008325C10013050900EF20C07FEF20907D94
:10186000832784046346F0026F0000031305090018
:10187000EF20502B63040500EF20105883278404C9
:101880009387F7FF2324F404832784046356F0002E
:1018900083274402E39C07FC23249404EF20D07C9C
:1018A000EF205079832744046346F0026F00000361
:1018B00013050A00EF20102763040500EF20D05322
:1018C000832744049387F7FF2322F40483274404E7
:1018D0006356F00083270401E39C07FC2322940451
:1018E000EF209078EF10501F63040508EF209074EC
:1018F00083278403E38E07F2938509001305040010
:101900008324C400EFE05FF163940A088327840313
:10191000032704009387F7FF232CF40263160700C4
:10192000EF20D07B2322A4008327040163920708C1
:10193000EF209073130510008320C103032481035B
:1019400083244103032901038329C102032A81025D
:10195000832A41021301010467800000EF20906D8B
:1019600003254400EF201050EF2010706FF05FEE61
:10197000EFE01FC26FF09FF783270504E38407D8C9
:10198000737004306F000000737004306F0000004B
:101990008327440223269400E38C07F813054402AE
:1019A000EF205018E30605F8EFE09FBE6FF05FF8F8
:1019B00013050401EF20101793071000E31AF5F642
:1019C0006FF09FFE13050400EFE05FE8EF10D0100A
:1019D000130500006FF05FF663000506130101FFB9
:1019E000232481002320210123261100232291009A
:1019F000832445001389050013040500EF20D0421D
:101A00006380A404930600001306090093050000F8
:101A100013050400EFF05FCC93071000630CF50290
:101A20008320C10003248100832441000329010095
:101A30001301010167800000737004306F00000023
:101A40008327C40013051000938717002326F40092
:101A50006FF01FFD8327C400938717002326F4002F
:101A60006FF01FFC630805066386050C130101FE79
:101A7000232C8100232A91002328210123263101D0
:101A80002324410113040500232E1100130906002D
:101A900093890500EFE01FC483278403130A050020
:101AA00093040000639C070213050A00EFE01FC2C5
:101AB0008320C1010324810113850400032901014E
:101AC000832441018329C100032A810013010102FB
:101AD00067800000737004306F0000000326040468
:101AE000630406028325C40083274400B385C50030
:101AF0002326B40063E6F500832504002326B40002
:101B000013850900EF40805B832784031307F0FFF0
:101B10009387F7FF232CF402832744046384E702AE
:101B20008327440493041000938717002322F404AE
:101B30006FF09FF783270504E38A07F27370043080
:101B40006F000000832704016396070093041000D0
:101B50006FF09FF513050401EF20C07CE30805FE3C
:101B6000E30609FE930710002320F9006FF01FFE23
:101B70006306050883270504638A0508638407084C
:101B8000130101FE232C8100232A91002328210127
:101B90002324410113040500232E110023263101C3
:101BA000138A0500EFE01FB38327840313090500A0
:101BB00093040000638E07008329C40093050A0084
:101BC00013050400EFE05FC59304100023263401E1
:101BD00013050900EFE09FAF8320C10103248101B9
:101BE0001385040003290101832441018329C100D5
:101BF000032A810013010102678000007370043022
:101C00006F000000737004306F000000E38C07FE6B
:101C1000737004306F0000006316050073700430A9
:101C20006F000000130101FF23248100130405004D
:101C300023261100EF20104003248403EF20D0421C
:101C40008320C10013050400032481001301010156
:101C50006780000063160500737004306F00000099
:101C6000130101FF23261100232481001304050022
:101C7000EF20503C832784030324C4033304F4403F
:101C8000EF20903E130504008320C100032481004F
:101C90001301010167800000630605000325850329
:101CA00067800000737004306F0000006308050453
:101CB00097870300938707A503A747006304E504FC
:101CC00003A7C7006302E50803A74701630AE50607
:101CD00003A7C7016302E50603A74702630AE504F9
:101CE00003A7C7026302E50403A74703630AE502EB
:101CF00003A7C7036302E5026F40C033737004306B
:101D00006F0000001307000013173700B387E700C8
:101D100023A007006F400032130770006FF0DFFE52
:101D2000130760006FF05FFE130750006FF0DFFDD8
:101D3000130740006FF05FFD130730006FF0DFFC0A
:101D4000130720006FF05FFC130710006FF0DFFB3C
:101D50000325C504678000002326B50467800000C2
:101D6000034505056780000063080500032585031A
:101D70001335150067800000737004306F00000099
:101D8000630C0500832785030325C5033305F54050
:101D90001335150067800000737004306F00000079
:101DA000978703009387079603A70700630007043C
:101DB00003A787006308070403A707016308070454
:101DC00003A787016308070403A707026308070442
:101DD00003A787026308070403A70703630C07042C
:101DE00003A787036304070467800000130700004C
:101DF00013173700B387E70023A0B70023A2A7007B
:101E000067800000130710006FF09FFE130720008B
:101E10006FF01FFE130730006FF09FFD13074000A7
:101E20006FF01FFD130750006FF09FFC1307700049
:101E30006FF01FFC130760006FF09FFB9787030094
:101E40009387478C03A747006300E50403A7C700F7
:101E50006306E50403A747016306E50403A7C7017A
:101E60006306E50403A747026306E50403A7C70268
:101E70006306E50403A74703630AE50403A7C70352
:101E80006302A704678000001307000013173700E0
:101E9000B387E70023A00700678000001307100046
:101EA0006FF0DFFE130720006FF05FFE13073000B6
:101EB0006FF0DFFD130740006FF05FFD1307500068
:101EC0006FF0DFFC130770006FF05FFC130760001A
:101ED0006FF0DFFB130101FF232481002322910017
:101EE00023202101130405002326110093840500FB
:101EF00013090600EF201014032744049307F0FF92
:101F00006314F70023220404032784049307F0FFDB
:101F10006314F70023240404EF201015832784039F
:101F2000639A070013060900938504001305440211
:101F3000EF20802EEF20101083278404635AF004D2
:101F40008327440263860704930444026F0000025F
:101F5000832784049387F7FF2324F40483278404CE
:101F60006358F00283274402638407021385040048
:101F7000EF20403BE30E05FCEF200068832784043C
:101F80009387F7FF2324F40483278404E34CF0FCB5
:101F90009307F0FF2324F404EF20100DEF209009A5
:101FA00083274404635AF0048327040163860704EB
:101FB000930404016F000002832744049387F7FF12
:101FC0002322F404832744046358F0028327040186
:101FD0006384070213850400EF20C034E30E05FC80
:101FE000EF208061832744049387F7FF2322F404C2
:101FF00083274404E34CF0FC9307F0FF2322F4040E
:10200000032481008320C1008324410003290100AF
:10201000130101016F20500597E701009387474A9C
:1020200083A6070017E701001307474803270700A7
:1020300023A2A600636AE504130101FF23248100A3
:102040002326110017E70100130747471304050073
:102050000325070083A5070093854500EFE08FF275
:1020600097E701009387C74283A707006376F400D0
:1020700097E7010023AE87408320C100032481003D
:10208000130101016780000017E701001307C74231
:102090000325070083A50700938545006FE08FEEB9
:1020A00097E701009387C74103A7070083A60700AE
:1020B000832747049387F7FF2322F70483A7460467
:1020C00063940700736004306780000063020504B6
:1020D000130101FD232E3101232A51012326110270
:1020E000938A0700232481022322910223202103C3
:1020F000232C41012328610123267101930740000D
:102100009309070063FAE700737004306F00000062
:10211000737004306F000000130B050093840500FA
:1021200013090600938B0600130A08006302082CAB
:1021300013050006EF301058130405006302052A4A
:102140001319290023284503130609009305500A93
:1021500013050A00EF40800803C704008327040327
:102160001309C9FF230AE40203C7040033892701C6
:102170001379C9FF6306070E83C71400A30AF4028C
:1021800083C71400638E070C83C72400230BF4025B
:1021900083C724006386070C83C73400A30BF402B3
:1021A00083C73400638E070A83C74400230CF402FC
:1021B00083C744006386070A83C75400A30CF40254
:1021C00083C75400638E070883C76400230DF4029D
:1021D00083C764006386070883C77400A30DF402F5
:1021E00083C77400638E070683C78400230EF4023E
:1021F00083C784006386070683C79400A30EF40296
:1022000083C79400638E070483C7A400230FF402DE
:1022100083C7A4006386070483C7B400A30FF40236
:1022200083C7B400638E070283C7C4002300F4048D
:1022300083C7C4006386070283C7D400A300F404E5
:1022400083C7D400638E070083C7E4002301F4042E
:1022500083C7E4006386070083C7F400A301F40486
:10226000130A440013050A00A301040423263403BF
:1022700023283405232A0404EFE04FCD13058401FD
:10228000EFE0CFCC93075000B3873741232C0404F1
:1022900023288400232CF400232284022322040414
:1022A000232E040413860B0093050B00130509006D
:1022B000EFE00FC32320A40063840A0023A08A0058
:1022C0007370043017E901001309C91D8327090041
:1022D00097E401009384C41E638C070003A70400E5
:1022E00083A7040083274704938717002322F7045A
:1022F00017E701001307C71B832707009387170001
:1023000097E6010023A6F61A83A70400638E070E42
:1023100083270900639C070083A7040083A7C702E3
:1023200063E6F90097E7010023AC871897E70100FF
:102330009387471603A7070097E601009386C61602
:102340008327C40283A606001307170017E60100BF
:102350002322E6142324E40463F6F60017E70100C1
:102360002324F71413074001B387E70217E50100A0
:102370001305052593050A003305F500EFE08FBD31
:10238000832709006388070083A7040083A7470405
:10239000639007128327090013041000638A070063
:1023A00083A7040083A7C70263F43701EFE04F9EC1
:1023B000130504008320C102032481028324410207
:1023C000032901028329C101032A8101832A4101D2
:1023D000032B0101832BC10013010103678000005F
:1023E00013050A00EF3010451304F0FF6FF05FFC97
:1023F00013152600EF30102C130A0500E31A05D23E
:102400001304F0FF6FF0DFFA97E7010023AA870AB1
:102410000327070093071000E31AF7F017E5010000
:102420001305051AEFE08FB017E501001305851AB3
:10243000EFE0CFAF17E501001305051BEFE00FAF8D
:1024400017E501001305851BEFE04FAE17E501000E
:102450001305051CEFE08FAD17EB0100130B8B1C70
:1024600013050B00EFE08FAC97EA0100938ACA1CBA
:1024700013850A00EFE08FAB17E501001305051D7A
:10248000EFE0CFAA17E501001305851DEFE00FAAC5
:1024900017E501001305051EEFE04FA997E70100BE
:1024A00023AE670197E7010023A857016FF01FE8EB
:1024B00003A7040083A60400832747049387F7FF3C
:1024C0002322F70483A74604E39607EC73600430E5
:1024D0006FF05FEC130101FF23248100232611001C
:1024E000232291002320210113040500737004307E
:1024F00097E40100938404FB83A70400639E071004
:102500006318040097E70100938787FB03A4070083
:102510001309440013050900EFE00FAC8327840280
:102520006386070013058401EFE00FAB93050900F4
:1025300017E501001305C512EFE0CFA197E70100F1
:10254000938747F703A7070097E70100938787F46E
:1025500083A707001307170097E6010023ACE6F4F2
:1025600003A704009387170097E6010023A4F6F25F
:10257000630C070097E70100938787F403A7070020
:1025800003274704631C070E83A70400638A07061A
:1025900097E701009387C7F203A70700630287103C
:1025A0007370043003A704006318070817E70100DD
:1025B0001307C7F08326070083A606006392060A66
:1025C0001307F0FF97E6010023A4E6EC03A704003D
:1025D0006308070203A707000327470463020702F3
:1025E00003A7070083A60700832747049387F7FF05
:1025F0002322F70483A74604639407007360043022
:102600008320C100032481008324410003290100A9
:10261000130101016780000097E70100938747EAF3
:1026200003A7070083A707008327470493871700A2
:102630002322F7046FF0DFEC83A6070003A707004F
:1026400003A746041307170023A2E60417E70100B7
:102650001307C7E68326070083A60600E38206F673
:10266000032707000327C7000327C70003274700E6
:1026700097E6010023AEE6E06FF05FF503A70700E1
:1026800083A60700832747049387F7FF2322F704D5
:1026900083A74604E39A07EE736004306FF0DFEE21
:1026A00097E70100938787DE83A70700638607000B
:1026B000737004306F000000032481008320C10088
:1026C0008324410003290100130101016FD05FEC55
:1026D0006304050C17E70100130787DE8326070054
:1026E000930700006386A60A130101FF2326110049
:1026F00023248100232291007370043097E60100A7
:10270000938646DA83A70600638C0700032607003A
:102710008327070083274604938717002322F604A4
:1027200083A706009304050003244501638807007E
:102730008327070083A747046394070697E70100F0
:102740009387C7D783A70700638C870697E70100A5
:10275000938787D683A707006384870697E70100DE
:10276000938747F16306F40497E70100938747EFE7
:10277000630CF402930710008320C100032481003E
:1027800083244100138507001301010167800000C5
:102790001385070067800000737004306F0000002D
:1027A000EFF01F906FF09FF9930740006FF0DFFC90
:1027B00083A7840293B71700938727006FF0DFFB8E
:1027C000930720006FF05FFB7370043097E7010000
:1027D000938747CD03A70700631607026304050428
:1027E00083A707000325C502638C070097E7010054
:1027F000938707CD03A7070003274704631C07023D
:102800006780000017E70100130787CB83260700C6
:102810000327070003A746041307170023A2E604B3
:10282000E31005FC17E70100130787C9032507001C
:102830006FF01FFB03A7070083A607008327470449
:102840009387F7FF2322F70483A74604E39A07FA46
:102850007360043067800000130101FF23248100AE
:102860001304050023261100EFD0DFE663180400EF
:1028700097E701009387C7C403A407000324C40299
:10288000EFD0DFE48320C10013050400032481009E
:1028900013010101678000009307400063F6B70051
:1028A000737004306F000000130101FE232C8100BF
:1028B000232E1100232A91002328210123263101F0
:1028C00023244101130405007370043017E901004B
:1028D000130949BD8327090063920710630004129E
:1028E00083270405638EF50A17E70100130747BD28
:1028F00063F0B70283260700638E86120327070062
:102900008324C702B3B4950093C414006F00000180
:1029100083240700B384844093B414000327C402C3
:102920006386E70E832784012328B40463C8070065
:1029300093075000B385B740232CB40093172700AA
:10294000B387E7000327440197E90100938949C74A
:1029500093972700B387F9006310F704130A440024
:1029600013050A00EFD05FE717E701001307C7B3AD
:102970008327C402032707006376F70017E70100E7
:102980002324F7B213074001B387E70293050A0037
:102990003385F900EFD01FDC63840400EFD05FBF04
:1029A00083270900638C070097E70100938747B1ED
:1029B00083A7070083A74704639E07048320C10100
:1029C0000324810183244101032901018329C100DA
:1029D000032A8100130101026780000097E70100CC
:1029E000938707AE03A7070083A707008327470441
:1029F000938717002322F704E31404EE97E70100FE
:102A0000938707AC03A407006FF09FED2326B40261
:102A10006FF05FF1032481018320C1018324410110
:102A2000032901018329C100032A81001301010246
:102A30006FF00FE7930400006FF05FEE630A050884
:102A4000130101FE232A910097E40100938444A717
:102A500083A70400232E1100232C810023282101A9
:102A6000232631016388A7047370043017E901003D
:102A7000130949A383270900638C070003A70400F7
:102A800083A7040083274704938717002322F704B2
:102A90000327450197E701009387C7BD630EF7023F
:102AA000832709006388070083A7040083A74704DE
:102AB000639E07088320C10103248101832441010F
:102AC000032901018329C10013010102678000006D
:102AD000737004306F0000008327850217E7010040
:102AE0001307C7B6E38EE7FAE39C07FA930945009C
:102AF0001304050013850900EFD01FCE17E701006E
:102B00001307879A8327C402032707006376F70019
:102B100017E70100232AF79813074001B387E7025C
:102B200017E501001305C5A9938509003305F500D4
:102B3000EFD05FC283A704000327C40283A7C702A4
:102B4000E360F7F6EFD0DFA46FF09FF50324810177
:102B50008320C10183244101032901018329C1008C
:102B6000130101026FF0CFD363020506130101FECA
:102B7000232C8100232A910023282101130405001E
:102B8000232E110023263101EFD0DFB403274401A7
:102B900097E70100938707AE13090500930400002F
:102BA000630AF70213050900EFD05FB28320C10169
:102BB00003248101138504000329010183244101B9
:102BC0008329C10013010102678000007370043083
:102BD0006F0000008327840217E50100130505A795
:102BE000E382A7FCE39007FC97E701009387078A3D
:102BF00083A707006394070697E701009387478C34
:102C000083A707008324C4029309440083A7C70253
:102C100013850900B3B4F400EFD01FBC17E701001F
:102C2000130787888327C4020327070093C414006F
:102C30006376F70017E701002328F78613074001A2
:102C4000B387E70217E5010013058597938509000F
:102C50003305F500EFD01FB06FF0DFF4930584016A
:102C6000EFD05FAF6FF01FF4130101FE37150000C6
:102C7000232E1100232C8100232A910023282101D7
:102C8000232631012324410123225101EF308022E8
:102C9000630605249304050013050006EF30802128
:102CA0001304050063000528371600009305500A39
:102CB0002328950213850400EF3040528324040337
:102CC000B71700009387C7FFB384F400B7474C459C
:102CD0009387974493094400232AF402138509003B
:102CE000230C0402A3010404232604022328040461
:102CF000232A0404EFD09FA513058401EFD01FA55C
:102D000093075000232C040493F4C4FF2328840069
:102D1000232CF4002322840223220404232E0404FF
:102D20001306000097150000938585EA13850400BB
:102D3000EFD01F9B2320A4007370043017D901002B
:102D4000130949768327090097D4010093844477B7
:102D5000638C070003A7040083A7040083274704AC
:102D6000938717002322F70417D70100130747742E
:102D7000832707009387170097D6010023AAF672CE
:102D800083A704006388070A83270900639C070060
:102D900083A7040083A7C7026396070097D70100A3
:102DA00023A0877297D701009387C76E83A7070078
:102DB00097D601009386466F0327C40283A60600B8
:102DC0009387170017D601002326F66C2324F404FA
:102DD00063F6E60097D7010023A8E76C9317270056
:102DE000B387E7009397270017D501001305457DAA
:102DF0003305F50093850900EFD0DF95832709009F
:102E00006388070083A7040083A74704639A070E1B
:102E1000832709006384070083A70400EF201006BE
:102E2000930710006304F512631A050A73700430E7
:102E30006F00000097D7010023A4876803270700CD
:102E400093071000E310F7F617D501001305457737
:102E5000EFD0DF8D17D501001305C577EFD01F8D9B
:102E600017D5010013054578EFD05F8C17D5010009
:102E70001305C578EFD09F8B17D501001305457951
:102E8000EFD0DF8A97DA0100938ACA7913850A00A6
:102E9000EFD0DF8917DA0100130A0A7A13050A0056
:102EA000EFD0DF8817D501001305457AEFD01F88D2
:102EB00017D501001305C57AEFD05F8717D501003C
:102EC0001305457BEFD09F8697D7010023A8575F56
:102ED00097D7010023A2475F6FF0DFEC8320C10189
:102EE0000324810183244101032901018329C100B5
:102EF000032A8100832A4100130101026780000038
:102F000003A7040083A60400832747049387F7FFE1
:102F10002322F70483A74604E39C07EE7360043082
:102F20006FF01FEF032481018320C10103290101F8
:102F30008329C100032A8100832A410013850400EC
:102F400083244101130101026F30C00E73700430FD
:102F50009307F0FF17D70100232CF75203248101B8
:102F600097D7010023A0A7548320C10183244101E6
:102F7000032901018329C100032A8100832A41001A
:102F800097D7010023A40752130101026FD08FC508
:102F90007370043097D7010023A607506FD0CFD6A7
:102FA00017D701001307874E832707009387170061
:102FB0002320F700678000007370043097D701006A
:102FC0009387474E03A707006318070217D701002E
:102FD0001307C74D0325070083A70700638C07006D
:102FE00097D701009387C74D03A70700032747041E
:102FF000631407026780000017D701001307474CCE
:10300000832607000327070003A7460413071700BA
:1030100023A2E6046FF09FFB03A7070083A6070027
:10302000832747049387F7FF2322F70483A74604E7
:10303000E39207FC7360043067800000130101FF16
:103040002326110023248100EFD0CFE897D7010079
:103050009387C74503A40700EFD04FE78320C10043
:10306000130504000324810013010101678000009F
:1030700097D701009387C74303A507006780000027
:10308000130101FD23261102232481022322910230
:1030900023202103232E3101232C4101232A510116
:1030A000232861012326710197D701009387073EEA
:1030B00083A70700639A070617D701001307073F86
:1030C000832707009387170097D6010023A0F63EB9
:1030D000832A0700638A0A0A97D701009387473B30
:1030E00083A707009304000063FEFA0A97D9010042
:1030F0009389094D17DA0100130A8A3C83270A00D5
:103100009306100003A7C70293172700B387E700B1
:1031100093972700B389F90083A7090063F4F602A7
:10312000930410006F00000297D701009387473780
:1031300083A70700930400009387170017D70100A7
:103140002320F73697D701009387473583A70700D9
:1031500063840700930410008320C10203248102CA
:103160001385040003290102832441028329C1013C
:10317000032A8101832A4101032B0101832BC10012
:10318000130101036780000017D401001304043306
:103190008327040083A707006388070C737004303B
:1031A0006F00000017D401001304443197D90100C7
:1031B0009389094117DA0100130A8A3017DB0100ED
:1031C000130B8B2E8327040083A707006380070857
:1031D0008327040083A7C70003A9C70083274900EA
:1031E000930B490013850B0063EAFA06EFD0CFDE9C
:1031F000832789021305890163840700EFD0CFDD9F
:103200008327C90203270B0093850B001395270022
:103210003305F500131525003385A9006376F70003
:1032200017D701002322F728EFD0CFD283270A0037
:103230000327C90283A7C702E366F7F883270400C0
:103240009304100083A70700E39407F89307F0FFA7
:1032500017D70100232EF7226FF05FEA17D701007E
:103260002328F7226FF09FE917D701001307C7241F
:10327000832704000327070097D6010023A0E62434
:1032800017D70100232AF72297D701009387C72079
:1032900083A707009387170017D70100232EF71E77
:1032A0008327040083A70700639A07009307F0FFB2
:1032B00017D70100232EF71C6FF01FE283270400AD
:1032C00083A7C70083A7C70083A7470017D70100BC
:1032D0002320F71C6FF05FE097D701009387071B4F
:1032E00003A7070063160700737004306F00000027
:1032F000130101FE232E1100232C8100232A9100AB
:1033000023282101232631012324410123225101B5
:10331000232061017370043097D4010093848418D2
:1033200003A704006310071203A707001307F7FFA2
:1033300097D6010023ACE61483A70700639E070A13
:1033400097D701009387C71683A707006386070AEC
:1033500097DA0100938ACA2617DA0100130ACA1401
:1033600017D901001309C915930910006F00C00196
:103370003385EA00EFD00FBE832709000327C4027C
:1033800083A7C7026374F70683A7CA086380070E82
:1033900083A78A0903A4C70013058401EFD0CFC314
:1033A000130B440013050B00EFD00FC38327C40297
:1033B00083260A0093050B00139527003305F500BB
:1033C00013152500130705003385AA00E3F2F6FA6A
:1033D00017D70100232AF70CEFD0CFB783270900B6
:1033E0000327C40283A7C702E360F7FA97D7010057
:1033F00023A6370B6FF05FF91304000083A70400C6
:10340000638C070097D701009387870B83A707007A
:1034100083A7470463980704130504008320C101B0
:103420000324810183244101032901018329C1006F
:10343000032A8100832A4100032B010013010102AA
:103440006780000017D7010013078707832607004E
:103450000327070003A746041307170023A2E60467
:103460006FF09FECEFE0DFC36FF01FFB17D401009C
:103470001304040383270400638C070283270400DA
:103480001309100063860702EFF09FBF6306050073
:1034900097D7010023A42701832704009387F7FF10
:1034A00017D70100232EF7FE83270400E39E07FCB5
:1034B00097D70100938787FE03A7070093071000A3
:1034C000E31CF7F2EFD0CF8C130410006FF01FF362
:1034D0006304050263960500737004306F000000FA
:1034E00017D70100130787FA83270700638A0700AD
:1034F000737004306F000000737004306F000000C0
:10350000130101FF232481002326110083260700D5
:10351000032705009386160017D601002328D6F648
:1035200097D60100938686F883A606003304B70079
:103530002320850063F0E6046372E40263F08602F0
:1035400097D701009387C7F703A507001305450028
:10355000EFD08FA813050400EFE01FACEFF0DFD72A
:10356000630E05008320C1000324810013010101C3
:1035700067800000E366E4FC6FF05FFC03248100D9
:103580008320C100130101016FD08F80630E0500FD
:1035900017D70100130787EF832707006388070009
:1035A000737004306F0000006FC09FFE130101FFB5
:1035B0002326110023248100032707009307050019
:1035C0001307170097D6010023A2E6EC97D6010057
:1035D000938606EF17D70100130747ED032707006F
:1035E00003A506003304F70013054500EFD0CF9E76
:1035F00013050400EFE05FA2EFF01FCE631A050091
:10360000032481008320C100130101016FC05FF812
:103610008320C100032481001301010167800000A1
:10362000130101FF232481002326110097D70100F5
:103630009387C7E583A7070013040000938717004B
:1036400017D701002324F7E497D70100938747E6B3
:1036500083A7070063ECF50E17DE0100130ECEFB07
:1036600097D20100938202F51304000013070000B3
:10367000930F10001303500A6F00C000130ECEFE0C
:103680006386C21183278EFF93050700E38807FE38
:103690008327CEFF83A74700232EFEFE6388C72122
:1036A00003AFC70083A747003307E500930E000070
:1036B000232EFEFE6380C70983A8C70093874803B3
:1036C000232017012322F70083A788042326F7016C
:1036D0002324F70083A7C8022328F70083A708053F
:1036E000232C0700232AF70003A8080383470800B8
:1036F000639A6706930708009387170083C607003D
:10370000B3850741E38A66FE93D5250093950501AD
:1037100093D50501231EB700938E1E0013070702E1
:10372000630C1F058327CEFF83A74700232EFEFED1
:10373000E394C7F983274E00232EFEFE6FF0DFF7D8
:10374000330464006304060023200600EFF0DFB8B2
:10375000130504008320C10003248100130101012B
:103760006780000093050000231EB700938E1E00A3
:1037700013070702E3181FFB3304D4011317540087
:10378000130ECEFE93050700E39EC2EF97D701000C
:103790009387C7D203AE070083270E00639E0710EE
:1037A00097D70100938747D103AE070083270E0008
:1037B0006392071C17DE0100130E8EE083270E0AAA
:1037C0006398072683274E0BE38E07F683278E0B1D
:1037D00097DE0100938E8EEA83A7470017D701007A
:1037E000232CF7E8638CD73D83AFC70083A747003E
:1037F0003307B5001303000097D6010023AEF6E6A9
:10380000130F3000930220009308500A6388D709F1
:1038100003A5C700930745032320A7002322F70031
:10382000832785042326E7012324F7008327C50285
:103830002328F70083278502638407002326570087
:1038400083270505232C0700232AF70003280503F7
:1038500083470800639C173393070800938717007A
:1038600083C60700B3850741E38A16FF93D5250079
:103870009395050193D50501231EB700130313008B
:1038800013070702E38EAFEA83278E0B83A7470057
:1038900097D6010023A2F6DEE39CD7F783270E0C10
:1038A00097D6010023AAF6DC6FF09FF683274E001F
:1038B000232EFEFE6FF0DFDE83274E00130F8E00F7
:1038C00083A647002322DE00638CE62DB307E500C4
:1038D00003A7460083A2C600930E00002322EE0039
:1038E000930F20001303500A6300EF088328C700DA
:1038F0001387480323A0170123A2E70003A7880426
:1039000023A6F70123A4E70003A7C80223A8E70022
:1039100003A7080523AC070023AAE70003A80803B0
:1039200003470800631A67221307080013071700EC
:1039300083460700B3050741E38A66FE93D5250059
:103940009395050193D50501239EB700938E1E0024
:1039500093870702638C122183264E0003A746003B
:103960002322EE00E314EFF80327CE002322EE001B
:103970006FF0DFF783274E00130F8E0083A74700F9
:103980002322FE006388E72183A2C70083A74700A4
:10399000B305B500930E00002322FE00930F200014
:1039A0001303500A6300FF0883A8C70093874803E6
:1039B00023A0150123A2F50083A7880423A6F501FF
:1039C00023A4F50083A7C80223A8F50083A7080550
:1039D00023AC050023AAF50003A8080383470800C9
:1039E00063946714930708009387170083C6070042
:1039F00033870741E38A66FE135727001317070131
:103A000013570701239EE500938E1E009385050240
:103A10006386121383274E0083A747002322FE00EC
:103A2000E314FFF88327CE002322FE006FF0DFF7B8
:103A300083274E0A17DF0100130F0FC383A7470028
:103A400017D701002320F7C26382E71783A2C700BC
:103A500083A74700B305B500930E000017D70100F8
:103A60002322F7C0930F40001303500A6382E70933
:103A700083A8C7009387480323A0150123A2F5005C
:103A800083A7880423A6F50123A4F50083A7C80211
:103A900023A8F50083A7080523AC050023AAF50099
:103AA00003A8080383470800639C67049307080082
:103AB0009387170083C6070033870741E38A66FEB2
:103AC000135727001317070113570701239EE5001B
:103AD000938E1E0093850502638E120383274E0A80
:103AE00083A7470017D70100232EF7B6E392E7F923
:103AF0008327CE0A17D701002326F7B66FF05FF7AA
:103B000013070000239EE500938E1E009385050297
:103B1000E39612FD83274E0B3304D4019315540012
:103B2000E38207C26FF09FCA13070000239EE500DF
:103B3000938E1E0093850502E39E12ED17DE0100B1
:103B4000130E0EA883270E0A3304D40193155400D4
:103B5000E38A07C66FF0DFED93050000239EB700F0
:103B6000938E1E0093870702E39812DF97D7010018
:103B70009387879403AE07003304D4019315540050
:103B800083270E00E38807C26FF0DFDE9305000095
:103B90006FF09FCE8327CE002322FE006FF0DFDE82
:103BA0008326CE002322DE006FF05FD28327CE0A69
:103BB00017D701002328F7AA6FF05FE983270E0CBF
:103BC00017D70100232AF7AA6FF01FC2130101FDC6
:103BD0002322910223202103232E3101232C410192
:103BE000232A510123286101232671012326110272
:103BF0002324810297D901009389498917D90100AB
:103C00001309099C17DA0100130ACA8997DA01001F
:103C1000938A0A8B97DB0100938B8B8997D40100E1
:103C200093844489130B10006F00000283A70900DE
:103C30000324090A9387170017D701002328F78464
:103C4000EFF08FE9631E040083A70400E39007FEF2
:103C500083270900E37AFBFEEFC09F936FF0DFFE3E
:103C60007370043083270A00639E07048327C90A00
:103C700003A4C70013054400EFC01FB683A70B00C1
:103C80009387F7FF17D701002324F78283A7040047
:103C90009387F7FF17D70100232EF78083270A00A9
:103CA0006388070083A70A0083A747046398070275
:103CB00003250403EF20003813050400EF208037AC
:103CC0006FF09FF803A70A0083A70A008327470421
:103CD000938717002322F7046FF05FF903A70A0008
:103CE00083A60A00832747049387F7FF2322F7045C
:103CF00083A74604E39E07FA736004306FF05FFB0E
:103D000097C701009387877883A707006396070EFC
:103D1000130101FF2326110097C7010023A0077894
:103D200017C701001307C77983270700B7A6A5A502
:103D30009386565A83A7070383A50700639ED50081
:103D400003A64700631AB60083A687006396C600E1
:103D500083A7C700638AD7000325070083250700D0
:103D600093854503EF30407697C601009386C6736E
:103D700003A6060017D70100130787846F0000020F
:103D800083A706006382070883A706009387F7FFCF
:103D900017C60100232AF67003A606009317260013
:103DA000B387C70093972700B307F70083A70700DF
:103DB000E38807FC03A6060093172600B387C70015
:103DC00093972700B305F70083A6450093878700E4
:103DD000B307F70083A6460023A2D500638AF60244
:103DE00083A7C6008320C10017C70100232AF76CF0
:103DF00013010101678000009307100017C701003D
:103E0000232EF76867800000737004306F00000095
:103E1000930740013306F60283A646003307C70026
:103E20002322D7006FF0DFFB130101FE23282101BD
:103E3000232E1100232C8100232A910023263101F7
:103E4000130905007370043097C4010093848465DE
:103E500083A7040017C4010013048466639C070C45
:103E6000631409000329040093094900138509001C
:103E7000EFC09F9683278902638607001305890197
:103E8000EFC09F959385090017C501001305857E36
:103E9000EFC05F8C83A704006388070083270400BA
:103EA00083A747046394070A832704006384270DCC
:103EB00083A70400638207067370043083A704009D
:103EC0006398070E97C701009387475F03A7070012
:103ED000032707006310070C9307F0FF17C70100C3
:103EE0002328F75A83A70400638807028327040066
:103EF00083A7470463820702032704008326040084
:103F0000832747049387F7FF2322F70483A74604F8
:103F100063940700736004308320C101032481018E
:103F200083244101032901018329C10013010102F6
:103F300067800000032704008327040083274704C9
:103F4000938717002322F7046FF09FF103270400E3
:103F500083260400832747049387F7FF2322F7046F
:103F600083A74604E39207F47360043083270400B8
:103F7000E39027F583A704006382070697C7010033
:103F80009387C75083A707006388070A73700430BC
:103F90006F00000083A7070083A7C70083A7C7009F
:103FA00083A7470017C701002324F74E6FF09FF344
:103FB00003270400832704008327470493871700FF
:103FC0002322F70497C701009387474F03A70700F1
:103FD00003270700E30207F06FF0DFFB97C701003C
:103FE0009387074D17C701001307875D83A7070055
:103FF0000327470B6314F7028320C10103248101C7
:1040000097C7010023AE074A832441010329010118
:104010008329C1001301010267800000032481018C
:104020008320C10183244101032901018329C100A7
:10403000130101026FF0DFCC032481018320C10151
:1040400083244101032901018329C10013010102D5
:104050006FC00FD46306050A130101FF23229100EC
:1040600097C401009384C4452320210113890500CE
:1040700083A5040023261100232481009385850154
:10408000EFC04FF003A5040013054500EFC0CFF4C7
:104090009307F0FF630AF90697C70100938707416A
:1040A00003A4070003A7040083A707003304240127
:1040B00023228700636EF40697C7010093870740A9
:1040C00003A5070083A5040093854500EFC08FEB8F
:1040D00097C701009387C73B83A707006376F40067
:1040E00097C7010023A6873A8320C10003248100DB
:1040F00083244100032901001301010167800000AE
:10410000737004306F00000083A504000324810055
:104110008320C100832441000329010017C5010049
:104120001305455593854500130101016FC08FE2CA
:1041300097C701009387473803A507000324810030
:1041400083A504008320C1008324410003290100CA
:1041500093854500130101016FC0CFE2630E050096
:1041600097C701009387873283A70700639A0700E8
:10417000737004306F000000737004306F00000033
:10418000130101FF2322910097C40100938444335B
:1041900003A704009387050083A50400B7060080E9
:1041A000B3E7D7002326110023248100232CF70036
:1041B0009385850113040600EFC0CFD903A5040041
:1041C00013054500EFC04FE19307F0FF6304F402CD
:1041D00097C701009387872D03A507008320C1009F
:1041E000832441003305850003248100130101016C
:1041F0006FD09FE283A50400032481008320C100C7
:104200008324410017C501001305C5469385450069
:10421000130101016FC00FD46308050A130101FFE8
:104220002322910097C40100938484292320210133
:104230001389050083A5040023261100232481008F
:104240009385850113040600EFC0CFD003A50400B9
:1042500013054500EFC04FD893071000630AF4061A
:1042600097C701009387872403A4070003A70400CE
:1042700083A707003304240123228700636EF4061A
:1042800097C701009387872303A5070083A5040030
:1042900093854500EFC00FCF97C701009387471F55
:1042A00083A707006376F40097C7010023A2871E47
:1042B0008320C100032481008324410003290100DD
:1042C0001301010167800000737004306F0000006B
:1042D00083A50400032481008320C10083244100BE
:1042E0000329010017C501001305C5389385450052
:1042F000130101016FC00FC697C701009387C71B49
:1043000003A507000324810083A504008320C100C6
:104310008324410003290100938545001301010115
:104320006FC04FC6130101FF232611002324810013
:10433000232291008327C50003A4C7006304040A55
:104340009304840113850400EFC00FC997C70100CF
:104350009387C71383A70700639A07089304440051
:1043600013850400EFC04FC797C701009387C71399
:104370000327C40283A7070063F6E70097C701007D
:1043800023A4E71293172700B387E700939727002A
:1043900017C501001305C522938504003305F500F8
:1043A000EFC04FBB97C701009387871183A7070012
:1043B0000327C4021305000083A7C70263FAE700BE
:1043C0009307100017C70100232AF70C13051000EC
:1043D0008320C100032481008324410013010101D3
:1043E00067800000737004306F0000009385040044
:1043F00017C5010013058525EFC0CFB56FF09FFAF3
:1044000097C701009387870883A707006396070073
:10441000737004306F000000130101FF23261100A8
:104420002324810023229100B70700800324C500C4
:10443000B3E7F5002320F50063080408EFC0CFB907
:104440009304440013850400EFC00FB997C701001F
:10445000938787050327C40283A7070063F6E70055
:1044600097C7010023A2E70493172700B387E7004B
:104470009397270017C50100130585143305F50030
:1044800093850400EFC00FAD97C7010093874703E2
:1044900083A707000327C4021305000083A7C702F0
:1044A00063FAE7009307100017C701002328F7FEFF
:1044B000130510008320C1000324810083244100E0
:1044C0001301010167800000737004306F00000069
:1044D0006304050297C70100938707FC03A7070041
:1044E00097C70100938787FC83A707002320E50077
:1044F0002322F50067800000737004306F00000015
:104500006304050E638E050C130101FF23261100C1
:1045100023248100130705007370043097C801003D
:10452000938848F883A708006380070297C70100B3
:10453000938707F983A6070083A7070083A746048C
:104540009387170023A2F60417C30100130303F691
:1045500083A70500032603009306F0FF1304000061
:104560006388D70417CE0100130E0EF303250E0047
:1045700003280700832647006306A80013041000E1
:104580006378D6023308D640130410006372F80231
:1045900003250E00B387C74003260300B387D70067
:1045A00023A0F5002320A7002322C7001304000046
:1045B00083A70800638C070097C70100938747F023
:1045C00083A7070083A74704639407021305040029
:1045D0008320C100032481001301010167800000D2
:1045E000737004306F000000737004306F000000BF
:1045F000EFD01FAB6FF09FFD9307100017C70100AE
:10460000232EF7E867800000630605000325C50434
:104610006780000013050000678000006304050048
:104620002326B5046780000097C70100938747E9F8
:1046300003A507006780000097C70100938787E6FE
:1046400083A7070013051000638C070097C70100BC
:104650009387C7E303A5070013351500131515004D
:1046600067800000630C0508130101FE232A9100F6
:1046700097C401009384C4E483A70400232E11008F
:10468000232C810023282101232631010327C50281
:1046900083A7C7026376F7048327850163CC0700ED
:1046A00083A7040083A6C70293075000B387D740AF
:1046B000232CF50093172700B387E7000327450154
:1046C00017C901001309C9EF93972700B307F90031
:1046D0006308F70283A7040083A7C7022326F50215
:1046E0008320C101032481018324410103290101A5
:1046F0008329C10013010102678000006780000068
:10470000930945001304050013850900EFC0CF8C01
:1047100083A7040017C70100130707D90327070061
:1047200083A7C7022326F4026376F70017C70100A8
:10473000232CF7D6139527003305F50003248101B8
:10474000131525008320C1018324410193850900AD
:104750003305A9008329C1000329010113010102C6
:104760006FB05FFF63060502130101FF23261100EE
:10477000232481002322910097C70100938747D407
:1047800003A40700630AA400737004306F000000E4
:104790001305000067800000832744056396070027
:1047A000737004306F0000008326C40203270405E1
:1047B0009387F7FF232AF4046384E600638E0700DF
:1047C000130500008320C1000324810083244100DD
:1047D0001301010167800000930444001385040065
:1047E000EFB09FFF8327040517C701001307C7CB4E
:1047F00083260700130750003307F7402326F402EF
:10480000232CE40063F6F60017C70100232EF7C837
:1048100013074001B387E70217C50100130545DA06
:10482000938504003305F500EFB0DFF213051000A7
:104830006FF05FF97370043097C70100938787C6E4
:1048400083A707006380070297C70100938747C7C4
:1048500003A7070083A70700832747049387170050
:104860002322F7046780000097C70100938787C35E
:1048700083A70700638C070297C70100938747C48B
:1048800003A70700032747046302070203A70700E3
:1048900083A60700832747049387F7FF2322F704A3
:1048A00083A74604639407007360043067800000A8
:1048B00097C701009387C7C003A6070083A6070018
:1048C00003A707009307500083A6C60203258601AD
:1048D000B387D740232CF7006780000097C70100FB
:1048E000938707BE03A70700630A070083A6070094
:1048F00003A746051307170023AAE60403A507002C
:1049000067800000130101FD2320210323261102EB
:104910002324810223229102232E31011309050051
:104920007370043097C401009384C4B783A7040054
:1049300017C401001304C4B8639E070A8327040048
:1049400083A78705639A07008327040013071000D5
:1049500023AEE704639A050E83A70400638807006B
:104960008327040083A74704639A071473700430F5
:1049700083A70400639407068327040003A5870523
:1049800063080500630209048327040023AC0704BD
:104990008327040023AE070483A70400638807006D
:1049A0008327040083A74704639207068320C1027C
:1049B0000324810283244102032901028329C101C6
:1049C0001301010367800000032704008327870584
:1049D0009387F7FF232CF7046FF09FFB0327040056
:1049E0008327040083274704938717002322F704B3
:1049F0006FF09FF8032704008327040083274704F0
:104A0000938717002322F7046FF05FF30327040056
:104A100083260400832747049387F7FF2322F704A4
:104A200083A74604E39407F8736004308320C1022F
:104A30000324810283244102032901028329C10145
:104A40001301010367800000032504002326B10041
:104A500013054500EFB05FD88325C1009307F0FF31
:104A60006380F50897C70100938747A483A90700CF
:104A70000327040083A70700B389B9002322370165
:104A800063ECF90697C70100938747A303A50700C6
:104A90008325040093854500EFB0DFCE97C7010062
:104AA0009387079F83A7070063F6F90097C7010064
:104AB00023A0379FEFB0DFAD6FF01FEA032704009C
:104AC00083260400832747049387F7FF2322F704F4
:104AD00083A74604E39C07E8736004306FF01FE986
:104AE0008325040017C501001305C5B8938545004B
:104AF000EFB05FC66FF01FFC97C701009387C79B9D
:104B000003A507008325040093854500EFB09FC7E8
:104B10006FF05FFA130101FD23202103232E3101E1
:104B2000232611022324810223229102232C4101F6
:104B300013890500930906007370043097C40100BF
:104B40009384449683A7040017C401001304449778
:104B5000639C071403270400930720000327C7055D
:104B60006304F702832704001345F5FF03A78705B5
:104B70003375E50023ACA704832704001307100056
:104B800023AEE704639A060A83A70400638807003C
:104B90008327040083A747046394071673700430C7
:104BA00083A70400639E0706638809008327040027
:104BB00083A7870523A0F9000327040093071000AB
:104BC000130500000327C705630EF70083270400C1
:104BD0001349F9FF1305100003A787053379E9008E
:104BE00023AC27058327040023AE070483A7040012
:104BF000638807008327040083A747046392070C98
:104C00008320C1020324810283244102032901027B
:104C10008329C101032A8101130101036780000078
:104C20000327040083270400832747049387170082
:104C30002322F7046FF05FF7032504002326D10039
:104C400013054500EFB05FB98326C1009307F0FF5D
:104C5000638AF60C97C701009387478503AA07006C
:104C60000327040083A70700330ADA002322470141
:104C70006368FA0C97C701009387478403A5070070
:104C80008325040093854500EFB0DFAF97C701008F
:104C90009387078083A707006370FA0A97B701001C
:104CA00023A8477F6F0040090327040083270400DF
:104CB00083274704938717002322F7046FF09FE9A7
:104CC0000327040083260400832747049387F7FF04
:104CD0002322F70483A74604E39407F273600430A9
:104CE0008320C1020324810283244102032901029B
:104CF0008329C101032A8101130101036780000098
:104D00000327040083260400832747049387F7FFC3
:104D10002322F70483A74604E39207E87360043074
:104D20006FF0DFE78325040017C5010013058594A4
:104D300093854500EFB01FA2EFB09F856FF0DFE4D1
:104D400097B701009387477703A5070083250400E1
:104D500093854500EFB01FA36FF01FFE630A050C9B
:104D6000130101FF23261100232481002322910037
:104D7000232021017370043097B40100938484725E
:104D800083A70400639607086386060083278505CA
:104D900023A0F60093070600930620000326C5050E
:104DA000232ED50413870500130405006382D70A58
:104DB00063F4F608930530006388B700930540005C
:104DC0006396B700630CD610232CE40493071000FD
:104DD000630CF6081304100083A70400638C07001B
:104DE00097B701009387C76D83A7070083A7470480
:104DF00063980706130504008320C1000324810083
:104E00008324410003290100130101016780000090
:104E100097B701009387C76A03A7070083A7070016
:104E200083274704938717002322F7046FF0DFF5E9
:104E3000737004306F00000093061000E398D7F8F9
:104E40008327850533E7B700232CE5046FF01FF8AF
:104E50008327850593871700232CF5046FF01FF730
:104E6000EFD00FA46FF01FF91309440013050900D8
:104E7000EFB09F9617B70100130707638327C4029B
:104E8000032707006376F70017B70100232EF760AA
:104E900013074001B387E70217B5010013054572F8
:104EA000930509003305F500EFB0DF8A83278402FC
:104EB00063860700737004306F00000097B701002D
:104EC0009387076083A707000327C40283A7C7024D
:104ED000E3F2E7F0EFB0CFEB6FF0DFEF1304000089
:104EE0006FF09FEF63080508130101FE232C81007A
:104EF000232A910023282101232631012324410163
:104F000023225101232E110093090700138A060062
:104F1000930406001389050013040500EFB08FFB0E
:104F2000930A050063060A00832784052320FA00FC
:104F30000327C40593072000232EF4046380F404A0
:104F400063FA9710930630006388D40093064000FC
:104F50006396D400630CF70E232C240593071000EE
:104F60006312F70A83278402638207027370043096
:104F70006F000000737004306F0000008327840509
:104F800093871700232CF4046FF05FFD97B701009F
:104F90009387C74F83A707006390070A93044400D1
:104FA00013850400EFB05F8317B701001307C74FE5
:104FB0008327C402032707006376F70017B70100B1
:104FC0002324F74E13074001B387E70217B501000A
:104FD0001305055F938504003305F500EFB08FF7E7
:104FE00097B701009387C74D83A707000327C40223
:104FF00083A7C70263F8E7006386090093071000E0
:1050000023A0F9001304100013850A00EFB00FEC81
:10501000130504008320C10103248101832441017D
:10502000032901018329C100032A8100832A410049
:1050300013010102678000009305840117B5010088
:105040001305C560EFB00FF16FF09FF91304000076
:105050006FF09FFB93071000E392F4F08327840521
:1050600033E92701232C24056FF05FEF630A050E57
:10507000130101FE232C8100232A91001304050053
:1050800023282101232E11002326310193840500BA
:10509000EFB04FE4930720008326C405232EF404C9
:1050A0008327840513071000130905009387170051
:1050B000232CF4046396E6088327840263860700A2
:1050C000737004306F00000097B701009387073CAE
:1050D00083A70700639A0708930944001385090012
:1050E000EFB08FEF17B701001307073C8327C40207
:1050F000032707006376F70017B701002326F73A66
:1051000013074001B387E70217B501001305454BAC
:10511000938509003305F500EFB0CFE397B70100A1
:105120009387073A83A707000327C40283A7C70210
:1051300063F8E700638604009307100023A0F400DF
:10514000032481018320C101832441018329C100FB
:105150001305090003290101130101026FB00FD7E4
:10516000737004306F0000009305840117B50100CF
:105170001305C54DEFB00FDE6FF05FFA9307050022
:10518000630805067370043017B7010013078731F1
:1051900083260700639E060203A6C7059306200028
:1051A000130500006316D60023AE07041305100094
:1051B00083270700638C070097B701009387473068
:1051C00003A7070003274704631C0702678000004A
:1051D00097B601009386C62E03A6060083A6060096
:1051E00083264604938616002322D6046FF0DFFA46
:1051F00097B701009387C72C83A707006FF09FF82C
:1052000003A7070083A60700832747049387F7FFB8
:105210002322F70483A74604E39A07FA7360043055
:1052200067800000130101FB232291042320210544
:10523000232C4103232A51032328610323267103CE
:105240002326110423248104232E310323248103E4
:10525000232291032320A10317B901001309492731
:1052600017BB0100130B0B2697B401009384C425D0
:1052700097BA0100938A8A25130A1000930B9000B5
:105280008327090003A707006306071683A7C70043
:1052900083A90700EFD0DFD0EFD01FD283270B0008
:1052A000130C05006368F50C97B7010023ACA72029
:1052B000130600006376352303A50400B3858941F6
:1052C000EFC05FC1EFE04F816306051603A5040040
:1052D000930600001306000093058100EFC0CFBFC6
:1052E000E30005FA83278100E3C207FE8329010159
:1052F00083A749016386070013854900EFB0CFCD2E
:10530000EFD09FCB83270B00130C05006362F50CD5
:105310008327810017B701002326871BE3E8FBFAE8
:10532000B317FA0013F707216310072013F7770C60
:105330006316072A93F70702E38A07F81385090023
:10534000EF00504F6FF09FF883A7C70003A4C7007A
:1053500083AC07009309440013850900EFB0CFC761
:105360008327440213050400E78007008327C40154
:105370006386470D8327090003A70700E31607FC90
:1053800003A70A0097B6010023AE861397B6010063
:1053900023AEF61297B7010023ACE712EFD0DFF38C
:1053A0006FF0DFF283A7C70003A4C70003AD0700B7
:1053B000930C440013850C00EFB00FC28327440206
:1053C00013050400E78007008327C401638C470BA3
:1053D0008327090003A70700E31607FC03A70A00B9
:1053E00097B6010023A4F60E97B7010023A2E70E9B
:1053F0006FF01FF2EFD0DFBAEFD01FBC83270B0096
:10540000130C0500E368F5F683A70A0003A5040062
:105410009309000003A60700B385894117B701006F
:105420002322870B13361600EFC0DFAAEFD0DFEA86
:10543000E31E05E8EFB0CF956FF05FE983278401A5
:1054400093850900B387FC0063E2FC0883A704008E
:1054500063860702232A0100232C9101232E810059
:10546000EFF08F9D03A504009306000013060000D3
:1054700093054101EFB00FECE31E05EE73700430AD
:105480006F0000008327840193850C00B307FD00A3
:105490006362FD0883A7040063860702232A0100D4
:1054A000232CA101232E8100EFF00F9903A5040006
:1054B000930600001306000093054101EFB08FE74B
:1054C000E31805F0737004306F0000000325090035
:1054D0002322F40023288400EFB0CFAA6FF09FE9C5
:1054E000EFD09FDF8327090083A7C70003A4C7006D
:1054F000930C440013850C00EFB00FAE8327C4015A
:10550000638A47058327440213050400E7800700E8
:105510006FF0DFDB032509002322F4002328840039
:10552000EFB04FA66FF0DFEA8327C10023ACF9008C
:105530006382070AB387870123A2F90023A83901F0
:10554000938549006362FC0803A50A00EFB08FA3AE
:105550006FF0DFD783278401232884003387F90085
:105560002322E400636AEC04330C3C41636EFC02CA
:1055700083A7040063860702232A0100232C31013C
:10558000232E8100EFF04F8B03A50400930600004B
:105590001306000093054101EFB0CFD9E31405F6DF
:1055A000737004306F00000003A50A0093850C009F
:1055B000EFB04F9D6FF01FF50325090093850C0098
:1055C000EFB04F9C6FF01FF403250900EFB08F9BE5
:1055D0006FF0DFCF737004306F0000008327C100CD
:1055E00083A6890123A839013387D70023A2E900C4
:1055F0006362EC06B307FC4063EAD70683A749025F
:1056000013850900E780070083A7C901E39047CD10
:1056100083A689018327C10003A70400B387D700AD
:1056200063060702232A0100232CF100232E3101F7
:10563000EFF08F8003A5040093060000130600001E
:1056400093054101EFB00FCFE31205C8737004302A
:105650006F0000006374FC00E372F7FA0325090091
:1056600093854900EFB00F926FF05FC603A50A0063
:1056700093854900EFB00F916FF05FC5130101FFF3
:1056800023248100232611002322910023202101BD
:1056900017B40100130444E3EFF0CF99832704000B
:1056A00063840704EFF04F9C83270400638A07029A
:1056B0009308000013080000930700001307200060
:1056C000930600001306004097B50100938505CFAF
:1056D00017050000130545B5EFC05F9F631405066D
:1056E000737004306F00000017B901001309C9F985
:1056F00013050900EFB08F8397B40100938404FA77
:1057000013850400EFB08F82130600009305C000DC
:105710001305400097B7010023AC27DB97B70100C2
:1057200023A697DAEFB00FAD17B70100232EA7D845
:105730006306050297B501009385C5C7EFC04FE624
:105740006FF05FF68320C1000324810083244100B1
:105750000329010013010101678000007370043008
:105760006F000000638A050A130101FD232A51011D
:10577000930A05001305C00223248102232291020B
:1057800023202103232E3101232C41012326110242
:10579000232861012326710113090700938906005C
:1057A000130A060093840500EF00C070130405007F
:1057B000630C0502EFF00F8897B701009387C7D0FD
:1057C00083A70700638E0704EFF00F8A13054400D8
:1057D00023205401232C9400232E4401232034033E
:1057E00023222403EFA09FF6130504008320C102A7
:1057F0000324810283244102032901028329C10178
:10580000032A8101832A4101032B0101832BC1005B
:105810001301010367800000737004306F00000003
:1058200097BB0100938B4BE613850B00EFA01FF095
:1058300017BB0100130B8BE613050B00EFA01FEF46
:10584000130600009305C0001305400097B7010040
:1058500023A077C997B7010023AA67C7EFB08F9934
:1058600017B701002322A7C6630A050097B50100F8
:10587000938545B4EFC0CFD26FF01FF5737004303D
:105880006F000000630E0506130101FE232C81004A
:10589000232E1100232A910017B401001304C4C25F
:1058A0008328040013080500130500006380080422
:1058B000930407002322B100138706002324C100AC
:1058C000232601019306500063C0B604EFE0DFD643
:1058D00093072000630EF5040325040093060000DF
:1058E0001306000093054100EFB0CFA48320C1014F
:1058F0000324810183244101130101026780000018
:10590000737004306F00000093054100930600009F
:105910001306070013850800EFB05FAE8320C101B6
:1059200003248101832441011301010267800000E7
:10593000032504009306000013860400930541002C
:10594000EFB04F9F6FF09FFA630605000325050037
:1059500067800000737004306F000000631605005C
:10596000737004306F000000130101FF2326110043
:105970002324810013040500EFE0DFEB032544013D
:105980003334A000EFE05FEE130504008320C10074
:1059900003248100130101016780000063160500E4
:1059A000737004306F000000130101FF2324810095
:1059B0001304050023261100EFE0DFE703240402AF
:1059C000EFE09FEA8320C100130504000324810057
:1059D0001301010167800000631605007370043035
:1059E0006F000000130101FF232481002322910096
:1059F000138405009304050023261100EFE09FE3C4
:105A000023A08402032481008320C1008324410059
:105A1000130101016FE05FE5130101FF1305C001F0
:105A20002324810023261100EF00C0481304050041
:105A3000630805002320050013054500EFA01FCFD4
:105A4000130504008320C100032481001301010118
:105A50006780000063020502B70700FFB3F7F50097
:105A600063860700737004306F000000639A0500BE
:105A7000737004306F000000737004306F0000001A
:105A8000130101FE232C810023282101232631014B
:105A90002324410123225101232E1100232A9100A6
:105AA0009309070013890600930A06001384050072
:105AB000130A0500EFE05FB863180500638609006C
:105AC000737004306F000000EFD08FCD83240A0084
:105AD000B3779400631209046382070463880A00A1
:105AE0009347F4FFB3F797002320FA00EFD0CFFEDF
:105AF0008320C101032481011385040003290101CE
:105B0000832441018329C100032A8100832A4100A3
:105B10001301010267800000E302F4FCE38809FC42
:105B2000B33550019395850163060900B70700045A
:105B3000B3E5F50013860900B3E5850013054A00B7
:105B4000EFE0CFE1EFD04FF963140500EFA05FA4C1
:105B5000EFE01FD6931765009309050063DA07008D
:105B6000B70400019384F4FFB3F499006FF05FF879
:105B7000EFE05FCC83290A00B37734016310090298
:105B8000638A070063880A009347F4FFB3F737017D
:105B90002320FA00EFE05FCD6FF09FFCE31CF4FEE2
:105BA0006FF05FFE630C0500B70700FFB3F7F50069
:105BB000638A0700737004306F0000007370043054
:105BC0006F000000130101FF23248100130405006E
:105BD000232611002322910023202101138905008F
:105BE000EFE05FC5832404009345F9FFB3F7950008
:105BF0002320F400EFE05FC78320C100032481006D
:105C000013850400032901008324410013010101CD
:105C100067800000130101FF2324810013040500A5
:105C200023261100EFA01FAB03240400EFA01FAA3E
:105C30008320C10013050400032481001301010126
:105C400067800000630C0500370700FFB3F7E5002D
:105C5000638A0700737004306F00000073700430B3
:105C60006F0000006F20501AB70700FFB377F600EF
:105C700063860700737004306F000000631606002F
:105C8000737004306F000000130101FE232C8100AB
:105C9000232821012326310123244101232E110031
:105CA000232A91001389060093890500130A050031
:105CB00013040600EFE05F98631E05046306090005
:105CC000737004306F000000EFD08FAD83240A00A2
:105CD0009385090013050A00B3E49900EFF09FF6DD
:105CE000B3779400630AF40883240A00EFD0CFDE70
:105CF0008320C101032481011385040003290101CC
:105D0000832441018329C100032A81001301010278
:105D100067800000EFD0CFA883240A009385090094
:105D200013050A00B3E43401EFF0DFF1B3F78400A8
:105D300063848704E30A09FAB7050005130609001E
:105D4000B365B40013054A00EFE04FC1EFD0CFD8E0
:105D500063140500EFA0DF83EFE09FB593176500A4
:105D60009304050063D40702B70700019387F7FF88
:105D7000B3F4F4006FF0DFF783270A001344F4FF55
:105D8000B3F787002320FA006FF05FF6EFE09FAAD9
:105D900083240A00B3779400639887009347F4FF45
:105DA000B3F797002320FA00EFE01FAC6FF0DFFBA2
:105DB000130101FF23248100232611001304050091
:105DC00023229100EFD0CF9D8327440063860702F2
:105DD000032504019304C400631895006F00800339
:105DE0000325040163089502B7050002EFE04FE1C7
:105DF00083274400E39607FE13050400EF00802389
:105E0000032481008320C100832441001301010188
:105E10006FD08FCC737004306F000000630C0500EE
:105E2000370700FFB3F7E500638A0700737004309B
:105E30006F000000737004306F0000006F20C07CA2
:105E4000630C0500B70700FFB3F7F500638A07008E
:105E5000737004306F000000737004306F00000036
:105E6000130101FF23248100232291002326110026
:105E70001304050093840500EFE0DF9B0327040073
:105E800093C7F4FFB377F7002320F40003248100C5
:105E90008320C10083244100130101016FE0DF9CD6
:105EA00063060500032585016780000013050000D7
:105EB00067800000130101FF2324810023261100C5
:105EC00013040500EFD0CF8D97A70100938787605B
:105ED00083A70700639C0704B797010017A7010079
:105EE0001307477D9387C7FF97A6010023AAE65EA5
:105EF00017A701002324F75E17A70100232EF77AC6
:105F000097A701009387475D17A701002324F77A1D
:105F10009307100017A701002326075C17A70100AD
:105F2000232C075A17A701002326F75A63120402ED
:105F3000EFD08FBAEF10805813040000130504004F
:105F40008320C10003248100130101016780000048
:105F500013058400937735006398070CB797010009
:105F60001307F5FF9387A7FFE3E4E7FC97A601007B
:105F70009386065783A706006F00400103A707001A
:105F8000630A0700938607009307070003A74700EB
:105F9000E366A7FE17A7010013070754E38AE7F893
:105FA00003A70700130600011384870023A0E6005F
:105FB00003A74700B306A740637ED6023388A70035
:105FC0002322D80023A2A7008325480097A601001A
:105FD000938606516F0080009306070003A7060012
:105FE00003264700E36AB6FE2320E80023A006014B
:105FF00003A7470097A701009387C75183A707000E
:10600000B387E74017A701002326F750EFD0CFACA6
:10601000E30204F2130504008320C100032481007D
:1060200013010101678000001375C5FF13054500CA
:106030006FF0DFF263080506130101FF23248100DE
:106040002326110013040500EFC09FF5930584FF7C
:106050000326C4FF17A70100130787486F008000BD
:10606000138707008327070083A64700E3EAC6FEDD
:10607000232CF4FE2320B70097A7010093878749BC
:1060800003A707008327C4FF032481008320C100E6
:10609000B387E70017A70100232EF746130101017C
:1060A0006FD08FA36780000097A701009387874672
:1060B00003A5070067800000678000003367B50014
:1060C0001377370093070500631207049308D6FF80
:1060D000B3081501130705009386050063781503BF
:1060E00003A806001307470093864600232E07FFE8
:1060F000E36817FF9347F5FFB387170193F7C7FFCF
:1061000093874700B385F500B307F5003306C50054
:1061100063F4C70C9386450013884700B3B6D700D5
:1061200033B8050133E7F50093C61600134818008D
:1061300013773700B3E60601133717003377D7001C
:10614000330EF64093861700630807061337AE0038
:106150006314070613532E00138805009386070067
:1061600013070000832808001307170013084800CE
:1061700023A0160193864600E36667FE1377CEFFE1
:10618000B385E500B387E7006306EE0483C6050028
:10619000138717002380D700637EC70283C61500CC
:1061A00013872700A380D7006376C70203C72500A3
:1061B0002381E70067800000B307F640B387F5004E
:1061C0009385150003C7F5FF93861600238FE6FE1F
:1061D000E398F5FE6780000067800000B367C500A4
:1061E00093F73700B308C5006382070E6376151175
:1061F000B307A04093F7370013873700930650008A
:1062000093F5F50F130815003383A8401306F6FF26
:106210006374D700130750006368E60E6380070EAF
:106220002300B50013071000638EE700A300B5003C
:1062300013073000130825006396E70013083500A4
:106240002301B5001396850033E6C50013970501B9
:106250003367E6003303F34093968501B366D700B6
:1062600013562300B307F5001307000023A0D7003F
:106270001307170093874700E36AC7FE1377C3FF2E
:10628000B307E8006300E3082380B7001387170013
:10629000637C1703A380B700138727006376170377
:1062A0002381B7001387370063701703A381B700FA
:1062B00013874700637A17012382B70013875700BB
:1062C00063741701A382B7006780000093F5F50F90
:1062D00013978500B365B700139705013367B700BF
:1062E000E37415FF930705009387470023AEE7FE8D
:1062F000E3EC17FF678000006780000013080500CB
:106300006FF05FF467800000930705006FF0DFF720
:106310008347050013070500638C0700130515006C
:1063200083470500E39C07FE3305E54067800000D6
:106330001305000067800000130515008347F5FF73
:106340009385150003C7F5FF63880700E386E7FE22
:106350003385E74067800000930700006FF05FFF20
:10636000930705009385150003C7F5FF9387170072
:10637000A38FE7FEE31807FE678000008346050051
:10638000930700026398F600130515008346050085
:10639000E38CF6FE938756FD93F7D70F63800704CF
:1063A00093070500930500006388060413050000A9
:1063B00093871700138606FD1317250083C6070071
:1063C0003305A700131515003305A600E39206FE5A
:1063D000638405003305A04067800000938536FD87
:1063E0008346150093B5150093071500E39006FC4E
:1063F000130500006FF0DFFD13050000678000004B
:1064000083A705002380A70083A7050093871700B3
:1064100023A0F5006780000097A601009386C60CB4
:1064200083A70600173703001307C7291386170031
:10643000B307F7002380A70097A5010023A6C50A8C
:106440009307A000630AF500930700046308F600B1
:106450001305000067800000E30C06FE370610F00D
:10646000130717008347F7FF2320F6F083A70600E2
:106470009387F7FF97A5010023A8F506E39207FE8F
:106480001305000067800000130101EB2322911423
:1064900023202115232A5113232481132326111489
:1064A00023248114232E3113232C41132328611319
:1064B00023267113232291132320A113232EB1111C
:1064C00093040500138905002326C100130C500214
:1064D000930A90008347090063888703638C07064B
:1064E00003A404006F008000638607062300F40005
:1064F00003A40400130919001304140023A084004A
:1065000083470900E39287FF0346190093081900A7
:1065100093860800130D00029309F0FF130AF0FFA1
:1065200013080000130550059307D6FD93F7F70FE6
:1065300013891600636EF53A17A70100130787AC9D
:1065400093972700B387E70083A70700B387E70087
:10655000678007008320C11403248114832441141D
:10656000032901148329C113032A8113832A4113A8
:10657000032B0113832BC112032C8112832C411294
:10658000032D0112832DC111130101156780000035
:10659000930C8000232401009307100063DA071D89
:1065A0008327C10003A40400938B770093F68BFF2D
:1065B00003AB060083A94600938786002326F100DB
:1065C00013860C009306000013050B009385090049
:1065D000EF1090422328A100930700006380373317
:1065E000930D4101930B100013860C0093060000DD
:1065F00013050B0093850900EF10C07C9306000083
:1066000013860C00130B050093890500EF10D03E94
:106610008327810023A0AD0093861B00938D4D003E
:1066200063863701938B06006FF01FFCE37C9BFFB2
:1066300063D24603930704002380A70103A4040048
:10664000130AFAFF9307140023A0F4001384070031
:10665000E3C446FF93962B0093070101B386D7004E
:106660006F008002938777052300F40003A40400E1
:10667000938BFBFF93871B001304140023A084005B
:106680009386C6FFE358F0E483A70600E3ECFAFC28
:10669000938707036FF05FFD83A704009306000351
:1066A0000327C1002380D70083A704009306470077
:1066B000930C00011386170023A0C4001306800763
:1066C000A380C70003A4040023240100930707004C
:1066D0001304140023A0840003AB070093090000F7
:1066E0002326D1006FF0DFED8327C10083AC0700C4
:1066F000938B470063880C28635C40259307D00286
:10670000631EFD2083C70C006388070263D8092439
:1067100083A60400938C1C00130AFAFF2380F60062
:1067200003A404001304140023A0840083C70C00F6
:10673000E39E07FC6352400303A404009307000296
:106740002300F40003A40400130AFAFF1304140046
:1067500023A08400E3160AFE232671016FF09FD761
:106760002324010093071000930CA000E3CA07E361
:106770008327C10003A40400938647006FF0DFF570
:1067800003C61600930609006FF01FDA83A7040002
:10679000930650022380D70003A4040013041400BE
:1067A00023A084006FF01FD3930C00012324010069
:1067B0006FF09FDE8327C10003C616009306090011
:1067C00083A90700938747002326F100E35E0AD4DC
:1067D000138A09009309F0FF6FF01FD503C6160056
:1067E000130DD002930609006FF01FD49347FAFFF0
:1067F00093D7F74103C61600337AFA0093060900CF
:106800006FF09FD203C61600130D00039306090014
:106810006FF09FD183C51600930906FD930609000A
:10682000938705FD13860500E3E2FAFA93972900A2
:10683000B38937019386160093991900B389B9007B
:1068400083C50600938909FD938705FD138605001E
:10685000E3FEFAFC6FF09FF70327C10083A7040053
:1068600083260700130747002326E1002380D70073
:1068700003A404001304140023A084006FF09FC538
:106880009307100063D4070F8327C1009386770016
:1068900093F686FF938786002326F10083A946009E
:1068A00083A7060063DE090E83A604001306D00248
:1068B000B307F0402380C60003A40400B336F00001
:1068C000B30930411304140023A08400138B070084
:1068D000B389D940930CA000232401006FF05FCE50
:1068E00003C6160013081800930609006FF0DFC3F3
:1068F00083A70400138908006FF09FE9E3729BCF20
:1069000093071000930B000093061000E3C447D3D5
:106910006FF05FD497AC0100938CCCAA93850900EB
:1069200013850C00EF104002330AAA406352400363
:1069300003A404002300A40103A40400130AFAFF23
:106940001304140023A08400E3160AFE130A0000B7
:1069500083C70C00E38207E0E3CC09DA9389F9FFEF
:106960001307F0FFE396E9DA6FF0DFDC8327C1005D
:106970009386470083A707002326D10093D9F741C8
:106980006FF05FF2635640019307D002E314FDF805
:1069900097AC0100938C0CA3930780026FF01FD774
:1069A000138B0700930CA0002324010003A4040010
:1069B0006FF01FC1130101EB232E3113B709004003
:1069C0009387F9FF2324811423229114232C41134C
:1069D000232A511323261114232021152328611360
:1069E0002326711323248113232291132320A1131F
:1069F000232EB111130A05002324B10017A40100AE
:106A0000130484AE973A0300938ACACB979401008B
:106A10009384C4742326F100930550021305A0004B
:106A200013080004B70610F083470A00638EB7040A
:106A30006388070A03270400130A1A0013061700C5
:106A40003387EA0097A8010023A0C8AA2300F70013
:106A50006380A708E31A06FD17370300130787C6EC
:106A6000130717008347F7FF23A0F6F083270400DE
:106A70009387F7FF17A601002328F6A6E39207FEE7
:106A800083470A00E396B7FA83461A0013051A00F3
:106A900013070500930B0002130BF0FF130CF0FF1C
:106AA0001308000093055005930890009387D6FDC6
:106AB00093F7F70F130A170063ECF5449397270039
:106AC000B387970083A70700B38797006780070005
:106AD00017370300130707BFE31406F86FF0DFF45E
:106AE0008320C11403248114832441140329011435
:106AF0008329C113032A8113832A4113032B011312
:106B0000832BC112032C8112832C4112032D0112FD
:106B1000832DC1111301011567800000930C8000C3
:106B2000130D00009307100063DA0721832781000B
:106B30009387770093F787FF83AD070003AB470088
:106B4000138787002324E10013860C0093060000BE
:106B500013850D0093050B00EF10006A2328A10098
:106B600063086D45130941019309100013860C0059
:106B70009306000013850D0093050B00EF10802491
:106B800013860C0093060000930D0500138B05007F
:106B9000EF1080662320A90093891900130949008A
:106BA000E3166DFDE3F49DFD13060004B70610F037
:106BB00063D489038327040013871700B387FA007F
:106BC00097A5010023A2E59223807701630AC706F7
:106BD000130CFCFFE3C089FF8327C1001305C1002C
:106BE00093089000B386F90093962600930701015D
:106BF000B386D7001308A00013030004370610F073
:106C0000E38CA6E083A706009305000363F4F80075
:106C10009305700503270400B387B7009305170099
:106C20003387EA0017AE01002320BE8C2300F70053
:106C300063860737638C65329386C6FF6FF05FFC0F
:106C400017370300130707A8130717008347F7FF39
:106C500023A0F6F0832704009387F7FF97A5010090
:106C600023A4F588E39207FE130CFCFF6FF09FF658
:106C700083270400130600041387170097A501005B
:106C800023A4E586B386FA00930500032380B600AB
:106C90006308C7509387270097A6010023A6F684B0
:106CA0003387EA00930680072300D70017370300D5
:106CB000130747A1B70610F06392C7021307170026
:106CC0008347F7FF23A0F6F0832704009387F7FF9D
:106CD00017A60100232AF680E39207FE832781008E
:106CE000930C0001130D00009387470003278100D8
:106CF000130B0000832D07002324F1006FF0DFE465
:106D00008327810083AC070013894700638E0C4CF6
:106D10006358802B9307D0026394FB3E03C70C009B
:106D2000930507006314072A6F00002F93071000D4
:106D3000930CA000130D0000E3CA07DF8327810036
:106D4000938747006FF09FFA8327810083461700DF
:106D500013070A0003AB0700938747002324F100C1
:106D6000E3560CD4130C0B00130BF0FF6FF01FD481
:106D700083461700930BD00213070A006FF01FD34E
:106D80009347FCFF93D7F74183461700337CFC0001
:106D900013070A006FF09FD183461700930B00037F
:106DA00013070A006FF09FD003461700138B06FDF0
:106DB00013070A00930706FD93060600E3E2F8FABC
:106DC00093172B00B38767011307170093971700DA
:106DD000B387C70003460700138B07FD930706FD23
:106DE00093060600E3FEF8FC6FF09FF78325810011
:106DF000832704001306A00003A70500938617004D
:106E0000B387FA00179501002320D56E2380E70091
:106E1000138945006300C736930700046384F62A8C
:106E2000232421016FF05FBF9307100063DE073555
:106E30008327810013877700137787FF93078700E5
:106E40002324F100032B47008327070063560B3EE2
:106E5000032704001306000493061700979501000A
:106E600023A4D5683387EA009305D0022300B70036
:106E7000638CC638B307F0403337F000330B604102
:106E8000938D0700330BEB40930CA000130D000013
:106E90006FF09FCB834617001308180013070A00F2
:106EA0006FF0DFC08346170013070A006FF01FC0A2
:106EB0008327040093060004138717001796010028
:106EC0002324E662B387FA00130650022380C7002A
:106ED000E314D7B4172703001307C77EB70610F0D3
:106EE000130717008347F7FF23A0F6F0832704005A
:106EF0009387F7FF179601002328F65EE39207FEBB
:106F00006FF09FB1930C0001130D00006FF09FC153
:106F10008327040093060004130A05001387170053
:106F2000179601002322E65CB387FA00130650028D
:106F30002380C700E312D7AE172703001307877813
:106F4000B70610F0130717008347F7FF23A0F6F0EA
:106F5000832704009387F7FF179601002326F6582E
:106F6000E39207FE130A05006FF01FAB172703001B
:106F700013074775130717008347F7FF2320F6F021
:106F8000832704009387F7FF9795010023AEF554FC
:106F9000E39207FE9386C6FF6FF09FC61727030094
:106FA00013074772E39805FC9386C6FF6FF05FC531
:106FB000E3FA9DBB930910006FF01FBF130C000094
:106FC00003C70C0093050700E30C07E49308F0FFE8
:106FD0001305A00013080004B70610F0635E0B0C45
:106FE0008327040013861700B387FA001793010064
:106FF000232CC34E2380E7006382A5086308060B99
:10700000938C1C0003C70C00130CFCFF93050700B6
:10701000E31607FCE35680E1832704009305000292
:1070200013060004B70610F06F00C000130CFCFF3D
:10703000E3080CDE13871700B387FA002380B7003C
:10704000179501002322E54A93070700E310C7FEC6
:107050001727030013070767130717008347F7FF76
:1070600023A0F6F0832704009387F7FF179501000C
:10707000232CF546E39207FE6FF05FFB1727030012
:1070800013074764E30E06F6130717008347F7FF5D
:1070900023A0F6F0832704009387F7FF17960100DB
:1070A0002324F644E39207FE6FF09FF517270300B1
:1070B000130747616FF05FFD130BFBFFE3121BF338
:1070C0006FF05FF5172703001307C75FB70610F0CF
:1070D000130717008347F7FF23A0F6F08327040068
:1070E0009387F7FF179601002320F640E39207FEEF
:1070F000232421016FF05F92979C0100938C8C2CCC
:1071000093050B0013850C00EF001004330CAC400A
:10711000E35880EB8327040013060004B70610F041
:107120006F00C000130CFCFFE30A0CE81387170084
:10713000B387FA00238077019795010023A6E53AEB
:1071400093070700E310C7FE1727030013078757AD
:10715000130717008347F7FF23A0F6F083270400E7
:107160009387F7FF9795010023A0F538E39207FE78
:107170006FF05FFB172703001307C754E39806F46B
:10718000232421016FF05F89832781001387470043
:1071900083A707002324E10013DBF7416FF01FCB27
:1071A0001727030013070752B70610F0130717003D
:1071B0008347F7FF23A0F6F0832704009387F7FFA8
:1071C000179601002322F632E39207FE9307100080
:1071D00017970100232AF73093078007172703002A
:1071E0002302F74E6FF09FAF635680019307D002E2
:1071F000E394FBF0979C0100938CCC1C1307800256
:10720000930580026FF09FDC972603009386864BE0
:10721000370610F09386160003C7F6FF2320E6F02A
:10722000032704001307F7FF9795010023AEE52A13
:10723000E31207FE6FF01FC4938D0700930CA000AC
:10724000130D00006FF05F90B70710F023A0A7F2B6
:107250006F000000130101FC130341022322B1025D
:1072600093050300232E11002324C1022326D102FB
:107270002328E102232AF102232C0103232E1103E8
:1072800023266100EFF00FF38320C10113050000F6
:107290001301010467800000130101FB1303810344
:1072A000232481022326A100232CC10213040500FC
:1072B000130603001305C100232611022322F10443
:1072C000232ED1022320E1042324010523261105C6
:1072D000232E6100EFF04F9B8327C100238007001E
:1072E0000325C1008320C1023305854003248102A8
:1072F0001301010567800000B70710F083A647F46B
:1073000003A607F403A747F4E31AD7FE9306067D06
:1073100033B6C600B305E60023A4D7F423A6B7F41A
:1073200067800000B70710F003A747F403A607F42F
:1073300083A647F4E31AD7FE9306067D33B6C6004C
:1073400023A4D7F4B305E60023A6B7F493070008F7
:1073500073A0473067800000130101FF23248100E0
:10736000232611009797010093878718179401002F
:107370001304C41703A707008327040093064706D6
:1073800093874706179601002322F616B7170000C9
:1073900017960100232ED614938777BB63CAD700B4
:1073A0008320C100032481001301010167800000D4
:1073B000B7F7FFFF9387C74A3307F7009797010096
:1073C00023A8E712EF008043930710006316F5022D
:1073D00003270400B72700009387773213050000C6
:1073E000E3D0E7FCEFF05FE6032481008320C100D7
:1073F000130101016FB0DFB917950100130505FDF9
:10740000EFF05FE513052000EFF01FE40324810097
:107410008320C100130101016FB09FB717950100D0
:10742000130585FC6FF01FE317950100130545FC5C
:107430006FF05FE2130101FF2324810023229100FA
:1074400023261100B7140000179401001304C4FA96
:1074500093878438130000009387F7FFE39C07FEAF
:1074600013050400EFF01FDF6FF09FFE13052000EF
:107470006F000015130101FF23261100EF000038F3
:107480001307100093070000631AE5008320C10072
:1074900013850700130101016780000017950100A3
:1074A0001305C5F2EFF01FDB8320C1009307200016
:1074B0001385070013010101678000007370043019
:1074C0006F00000067800000737004306F000000E0
:1074D000130101FE232C8100232A9100232821017E
:1074E000232E1100130405002317010013090000C7
:1074F000930410006F00800013091000032644005D
:1075000003250400930600009305E100EF905FB4AB
:10751000E31495FE631E09000327840083570700C8
:10752000938717009397070193D707412310F7001C
:107530008357E100938717002317F1006FF01FFCBA
:10754000130101FD23248102232291022320210320
:10755000232E310123261102130405009309000094
:1075600093040000130910000326440003250400BF
:10757000930600009305E100EF909FCCE31625FFF2
:107580008357E100638897009384070093091000F4
:107590006FF09FFD93841400639E0900032784000D
:1075A00083570700938717009397070193D70741E5
:1075B0002310F7009394040193D404016FF0DFFAD1
:1075C000130101FE23263101930905001305C000B4
:1075D000232E1100232C8100232A9100232821012E
:1075E000EFE05F8D130405001306000093052000F3
:1075F00013051000EF900FC01309803E979701000C
:107600009387C7F02320A400232224012324F4001D
:107610001305C000EFE01F8A930405000325040052
:10762000138709009306040023A0A4001795010006
:10763000130545ED23A4A4009308000013080000DF
:10764000930700001306004097950100938505DC21
:1076500023A20400170500001305C5EEEFA01FA725
:10766000938604009308000013080000130700002D
:10767000930700001306004097950100938585D974
:1076800017050000130505E5EFA05FA41305C00072
:10769000EFE05F821304050013060000930520004D
:1076A00013051000EF900FB5979701009387A7E59A
:1076B0002320A4002324F400232204001305C00087
:1076C000EFE04FFF93040500032504009306040038
:1076D00023A2240123A0A40017950100130525E38C
:1076E00023A4A400930800001308000093070000DF
:1076F000130700001306004097950100938505D2FB
:1077000017050000130505E4EFA05F9C138709002F
:1077100093860400930800001308000093070000FC
:1077200013060040979501009385C5CF170500000B
:10773000130545DAEFA09F991305C000EFE08FF71E
:1077400013040500130600009305200013055000E4
:10775000EF904FAA97970100938707DB2320A4009F
:10776000232224012324F4001305C000EFE08FF44A
:1077700093040500032504009306040023A22401BA
:1077800023A0A40017950100130585D823A4A40005
:10779000930800001308000093070000130700007F
:1077A0001306004097950100938545C81705000012
:1077B000130545D2EFA09F91032481018320C101CD
:1077C000032901018329C100938604008324410118
:1077D000930800001308000093070000130700003F
:1077E00013060040979501009385C5C41705000056
:1077F000130545D5130101026FA05F8D130101FF31
:1078000023222101232681002324910023203101FA
:1078100017950100130585CF17980100130888CE2E
:1078200083540500835E0500835908001799010001
:10783000130949CC035E0800035425008315090091
:1078400017970100130787CB035325008317070001
:1078500083532800031627009399090183582800B1
:1078600093D90941835245009394040113140401F0
:10787000035F450083162900835F480093D40441C9
:10788000B38535411354044103174700B38797402C
:1078900033068640B335B0009393030103154900C6
:1078A000B305B04093D30341B337F0003336C00083
:1078B00093920201B3F7B7003306C040B386764017
:1078C00093D2024193950F01B3F7C700B336D000AE
:1078D000035648003307574093D505410324C100A0
:1078E000B306D0403337E0003305B5403307E040FE
:1078F000B3F7D7003335A000B3F7E7003305A04056
:1079000017970100231CD7BF179701002314C7BF87
:1079100017970100231567BE17970100231D17BD98
:1079200017970100231EE7BD179701002316C7BC58
:1079300083248100032941008329010033F5A70036
:107940001301010167800000B305B500930705002E
:107950006386B70003C70700631607003385A74097
:1079600067800000938717006FF09FFE9308000068
:1079700063DC05003305A040B337A000B305B04079
:10798000B385F5409308F0FF63DA06003306C04084
:10799000B337C000B306D040B386F64013080600E4
:1079A00013830600930705001387050063980624D8
:1079B000979601009386069063F8C50E370E010076
:1079C000637AC60D130EF00F6374CE0013038000AC
:1079D000335E6600B386C60103CE0600330E6E002A
:1079E000130300023303C341630C0300B395650026
:1079F000335EC501331866003367BE00B3176500F8
:107A0000135E0801B355C70313150801135505018B
:107A100093D607013376C703B305B50213160601E3
:107A2000B366D60063FAB600B386060163E60601C4
:107A300063F4B600B3860601B386B64033F7C603D7
:107A40009397070193D70701B3D6C603B306D502B0
:107A500013150701B367F50063FAD700B387070171
:107A600063E6070163F4D700B3870701B387D74004
:107A700033D5670093050000638C0800B307A0406E
:107A80003337F000B305B04013850700B385E540F8
:107A900067800000370E000113030001E36AC6F39C
:107AA000130380016FF0DFF2631606001308100065
:107AB00033586802370701006372E80A1307F00FB2
:107AC000637407011303800033576800B386E60030
:107AD00003C6060033066600130300023303C340E7
:107AE00063180308B385054193560801131508016F
:107AF0001355050113D6070133F7D502B3D5D502C7
:107B0000131707013367C700B305B502637AB700DF
:107B100033070701636607016374B7003307070182
:107B2000B305B74033F7D5029397070193D7070101
:107B3000B3D5D502B305B50213150701B367F50038
:107B400063FAB700B387070163E6070163F4B70080
:107B5000B3870701B387B7406FF09FF13707000184
:107B600013030001E362E8F6130380016FF0DFF511
:107B70003318680033DEC500935E08013356C50034
:107B8000B31765003355DE03B39565003366B60061
:107B90009315080193D50501935606013377DE034B
:107BA0003385A502131707013367D700637AA7004F
:107BB00033070701636607016374A70033070701F2
:107BC000B306A74033F7D603131606011356060172
:107BD000B3D6D60313170701B386D502B365C70022
:107BE00063FAD500B385050163E6050163F4D500AA
:107BF000B3850501B385D5406FF01FEFE3EED5E601
:107C00003708010063FC0605930EF00F33B8DE0061
:107C10001318380033DE060117830100130383694C
:107C20003303C301834E0300130E0002B38E0E0113
:107C3000330EDE41631E0E0263E4B600636AC500C4
:107C4000B307C540B385D5403335F5003387A5402C
:107C500013850700930507006FF01FE2370300014B
:107C600013080001E3E866FA130880016FF09FFA39
:107C70003357D601B396C601B366D700B357D501C3
:107C800033D7D501B395C501B3E7B70093D5060146
:107C90003373B702139F0601135F0F0113D8070157
:107CA0003316C6013315C5013357B7021313030149
:107CB00033680301B30FEF0213030700637EF8017B
:107CC0003308D8001303F7FF6368D8006376F80120
:107CD0001303E7FF3308D8003308F841B37FB80235
:107CE0003358B802939F0F01B3050F03139F070189
:107CF000135F0F0133EFEF0113070800637EBF002E
:107D0000330FDF001307F8FF6368DF006376BF00FF
:107D10001307E8FF330FDF0013130301B70F010050
:107D20003363E3009387FFFF13580601330FBF400F
:107D3000B375F30013530301B377F6003387F502ED
:107D4000B307F302B385050333030303B385F500DB
:107D5000135807013308B8006374F8003303F301C4
:107D6000B70701009387F7FF935508013378F800B0
:107D7000131808013377F700B38565003307E8006F
:107D80006366BF00631EBF00637CE5003306C74027
:107D90003337C700B385D540B385E54013070600E8
:107DA0003307E5403335E500B305BF40B385A54053
:107DB000B397D5013357C70133E5E700B3D5C50104
:107DC0006FF09FCB9387050013080600138706000A
:107DD0001303050063960628978801009388884D51
:107DE00063F6C50E370701006378E60C1307F00F42
:107DF0003337C70013173700B356E600B388D800EF
:107E000083C608003387E60093060002B386E64087
:107E1000638C0600B397D7003357E5003318D600BC
:107E2000B365F7003313D50013550801B3D7A50286
:107E300013160801135606019356030133F7A502E2
:107E4000B305F60213170701B366D70013870700BF
:107E500063FEB600B38606011387F7FF63E80601E9
:107E600063F6B6001387E7FFB3860601B386B64014
:107E7000B3F7A6021313030113530301B3D6A602EB
:107E80009397070133E36700B305D6021385060015
:107E9000637CB300330368001385F6FF6366030158
:107EA0006374B3001385E6FF131707013367A70058
:107EB000930500006F00400EB70600011307000194
:107EC000E36CD6F2130780016FF01FF36316060010
:107ED0009306100033D8C602B70601006372D80CAF
:107EE0009306F00F63F4060113078000B356E80011
:107EF000B388D80083C60800B386E60013070002E3
:107F00003307D7406318070AB3870741930510006A
:107F1000135608019318080193D8080193560301DA
:107F200033F7C702B3D7C70213170701B366D700E9
:107F30003385F8021387070063FEA600B3860601A7
:107F40001387F7FF63E8060163F6A6001387E7FFD0
:107F5000B3860601B386A640B3F7C6021313030126
:107F600013530301B3D6C6029397070133E36700A7
:107F7000B388D80213850600637C130133036800BD
:107F80001385F6FF63660301637413011385E6FF2F
:107F9000131707013367A700130507006780000068
:107FA000B706000113070001E362D8F4130780014C
:107FB0006FF0DFF33318E800B3D5D7003313E500D3
:107FC000B356D50013550801B397E70033F7A50260
:107FD000B3E8F6009317080193D7070113D60801F9
:107FE000B3D5A502131707013367C700B386B702DD
:107FF00013860500637ED700330707011386F5FF5C
:10800000636807016376D7001386E5FF330707012E
:10801000B306D74033F7A6029398080193D8080116
:10802000B3D6A60213170701B385D702B3671701AA
:108030001387060063FEB700B38707011387F6FFB7
:1080400063E8070163F6B7001387E6FFB38707010C
:10805000B387B74093150601B3E5E5006FF05FEB1A
:1080600063E6D5183707010063F4E6041308F00F40
:108070003337D8001317370033D8E600978501004F
:1080800093854523B385050103C8050093050002C8
:108090003308E800B3850541639605021307100015
:1080A000E3ECF6EE3335C500134715006FF0DFEE55
:1080B000B705000113070001E3E0B6FC13078001D8
:1080C0006FF09FFB33570601B396B600B366D70037
:1080D00093DE060133D70701B378D703B397B70010
:1080E000335805013363F8009397060193D70701CE
:1080F000135803013316B6003357D703939808017A
:1081000033E80801338FE702130E0700637EE801AE
:108110003308D800130EF7FF6368D8006376E801D0
:10812000130EE7FF3308D8003308E841B378D803CB
:108130003358D80393980801B38E070393170301AC
:1081400093D70701B3E7F8001307080063FED701D0
:10815000B387D7001307F8FF63E8D70063F6D701AA
:108160001307E8FFB387D700131E0E01B387D7416B
:10817000B70E01003367EE001388FEFF337307016B
:10818000935807013378060113560601330E030393
:108190003388080393560E013303C30233030301EC
:1081A000B3866600B388C80263F40601B388D801B9
:1081B00013D60601B308160163E61703E39A17CF37
:1081C000B70701009387F7FFB3F6F6009396060111
:1081D000337EFE003315B500B386C601930500005B
:1081E000E37CD5DA1307F7FF6FF09FCC930500000F
:1081F000130700006FF05FDA93080600138706008C
:108200009307050013880500639C062297860100EA
:108210009386460A63FCC50C37030100637E660A39
:108220001303F00F6374C300130780003353E60099
:10823000B386660003CE060013030002330EEE0081
:108240003303C341630C0300B3956500335EC5017E
:10825000B31866003368BE00B317650013D6080173
:108260003377C802139508011355050193D607010A
:108270003358C80213170701B366D7003308050344
:1082800063FA0601B386160163E6160163F406017C
:10829000B3861601B386064133F7C60293970701EA
:1082A00093D70701B3D6C602B306D502131507014B
:1082B000B367F50063FAD700B387170163E61701C8
:1082C00063F4D700B3871701B387D74033D567006E
:1082D00093050000678000003703000113070001C9
:1082E000E36666F4130780016FF05FF4631606001F
:1082F00013061000B35816033706010063F2C80ACC
:108300001306F00F637416011307800033D6E800DC
:10831000B386C60003CE060013030002330EEE0040
:108320003303C34163180308B385154113D708010C
:10833000139508011355050113D60701B3F6E5029D
:10834000B3D5E50293960601B3E6C600B305B502C0
:1083500063FAB600B386160163E6160163F4B6004D
:10836000B3861601B385B640B3F6E50293970701CD
:1083700093D70701B3D5E502B305B50213950601FE
:10838000B367F50063FAB700B387170163E6170117
:1083900063F4B700B3871701B387B7406FF01FF3DB
:1083A0003706000113070001E3E2C8F61307800156
:1083B0006FF0DFF5B398680033D7C501B3176500D8
:1083C000335EC50113D50801B376A702B3956500E6
:1083D000336EBE009395080193D5050113560E0127
:1083E0003357A70293960601B3E6C6003387E5022A
:1083F00063FAE600B386160163E6160163F4E6004D
:10840000B38616013386E640B376A602131E0E012C
:10841000135E0E013356A602939606013386C502FB
:10842000B3E5C60163FAC500B385150163E615011E
:1084300063F4C500B3851501B385C5406FF01FEF28
:10844000E3EAD5E83707010063FCE604930EF00F7A
:1084500033B7DE001317370033D3E60097880100E7
:10846000938848E5B388680083CE0800130E0002A5
:10847000B38EEE00330EDE41631E0E0263E4B600DF
:10848000636AC500B307C540B385D5403335F500F1
:108490003388A54013850700930508006FF09FE31C
:1084A000B708000113070001E3E816FB130780017A
:1084B0006FF09FFA3357D601B396C601B366D70063
:1084C000B357D50133D7D501B395C501B3E7B7008D
:1084D00093D506013373B702139F0601135F0F0193
:1084E00093D807013316C6013315C5013357B702B8
:1084F00013130301B36813013308EF0213030700DA
:1085000063FE0801B388D8001303F7FF63E8D800BF
:1085100063F608011303E7FFB388D800B388084166
:10852000B3FFB802B3D8B802939F0F01B3051F037E
:10853000139F0701135F0F0133EFEF01138708004B
:10854000637EBF00330FDF001387F8FF6368DF002F
:108550006376BF001387E8FF330FDF0013130301B7
:10856000B70801003363E3009387F8FF135806014F
:10857000330FBF40B375F30013530301B377F60015
:108580003387F502B307F302B3850503330303030F
:10859000B385F500135807013308B8006374F80079
:1085A00033031301B70701009387F7FF93550801C1
:1085B0003378F800131808013377F700B3856500A6
:1085C0003307E8006366BF00631EBF00637CE500FD
:1085D0003306C7403337C700B385D540B385E54080
:1085E000130706003307E5403335E500B305BF4008
:1085F000B385A540B397D5013357C70133E5E700ED
:10860000B3D5C5016FF01FCD130101FE232C8100EE
:10861000232A9100130405009384050023282101D7
:10862000232631012324410123225101232E11004D
:10863000EFA01F978327040003290401B709000155
:10864000B3E59700930AC4002320B400930400000C
:108650009389F9FF370A00020327040063822A0581
:108660000326090013050900B3654701B3763601F7
:108670009317560033F7E6000329490063C6070045
:10868000631607006FF05FFDE398E6FC9317760032
:1086900063D40700B3E4D400EFB09FD66FF0DFFBE4
:1086A00093C4F4FFB3F4E40023209400EFA0DFC2EE
:1086B000032504008320C101032481018324410197
:1086C000032901018329C100032A8100832A410073
:1086D0001301010267800000130101FF1305200050
:1086E0002326110023248100EFE09FED17F7FFFF01
:1086F0001307C7C693060000130610009305400633
:10870000178501001305C5CFEFD0CF8563020502A1
:1087100013040500EFA05F8A13060500130700008D
:10872000930600009305100013050400EFD08F9509
:10873000EFA08FD38320C100032481001305000024
:08874000130101016780000034
:02000004800278
:100000008067FEFFF068FEFF8C67FEFFF068FEFF72
:10001000F068FEFFF068FEFFF068FEFFB467FEFFC9
:10002000F068FEFFF068FEFFDC67FEFFEC67FEFF96
:10003000F068FEFF0468FEFF1468FEFF1468FEFF10
:100040001468FEFF1468FEFF1468FEFF1468FEFFCC
:100050001468FEFF1468FEFF1468FEFFF068FEFFE0
:10006000F068FEFFF068FEFFF068FEFFF068FEFF3C
:10007000F068FEFFF068FEFFF068FEFFF068FEFF2C
:10008000F068FEFFF068FEFFF068FEFFF068FEFF1C
:10009000F068FEFFF068FEFFF068FEFFF068FEFF0C
:1000A000F068FEFFF068FEFFF068FEFFF068FEFFFC
:1000B000F068FEFFF068FEFFF068FEFFF068FEFFEC
:1000C000F068FEFFF068FEFFF068FEFFF068FEFFDC
:1000D000F068FEFFF068FEFFF068FEFFF068FEFFCC
:1000E000F068FEFFF068FEFFF068FEFFF068FEFFBC
:1000F000F068FEFFF068FEFFF068FEFFF068FEFFAC
:100100005868FEFF8068FEFFF068FEFFF068FEFFA3
:10011000F068FEFFF068FEFFF068FEFFF068FEFF8B
:10012000F068FEFFE068FEFFF068FEFFF068FEFF8B
:100130009065FEFF9866FEFFF068FEFFF068FEFF28
:10014000E866FEFFF068FEFF6067FEFFF068FEFFF6
:10015000F068FEFFA867FEFF4C6DFEFFB86DFEFF66
:10016000586DFEFFB86DFEFFB86DFEFFB86DFEFF67
:10017000B86DFEFFF06BFEFFB86DFEFFB86DFEFFC1
:10018000186CFEFF286CFEFFB86DFEFF406CFEFF92
:10019000506CFEFF506CFEFF506CFEFF506CFEFF7B
:1001A000506CFEFF506CFEFF506CFEFF506CFEFF6B
:1001B000506CFEFFB86DFEFFB86DFEFFB86DFEFF20
:1001C000B86DFEFFB86DFEFFB86DFEFFB86DFEFFA7
:1001D000B86DFEFFB86DFEFFB86DFEFFB86DFEFF97
:1001E000B86DFEFFB86DFEFFB86DFEFFB86DFEFF87
:1001F000B86DFEFFB86DFEFFB86DFEFFB86DFEFF77
:10020000B86DFEFFB86DFEFFB86DFEFFB86DFEFF66
:10021000B86DFEFFB86DFEFFB86DFEFFB86DFEFF56
:10022000B86DFEFFB86DFEFFB86DFEFFB86DFEFF46
:10023000B86DFEFFB86DFEFFB86DFEFFB86DFEFF36
:10024000B86DFEFFB86DFEFFB86DFEFFB86DFEFF26
:10025000B86DFEFFB86DFEFF946CFEFFD06CFEFF24
:10026000B86DFEFFB86DFEFFB86DFEFFB86DFEFF06
:10027000B86DFEFFB86DFEFFB86DFEFF3C6DFEFF72
:10028000B86DFEFFB86DFEFFC469FEFF186BFEFF80
:10029000B86DFEFFB86DFEFFA86BFEFFB86DFEFFE8
:1002A000D46BFEFFB86DFEFFB86DFEFFAC6DFEFFB8
:1002B000000102020303030304040404040404040D
:1002C00005050505050505050505050505050505DE
:1002D00006060606060606060606060606060606BE
:1002E00006060606060606060606060606060606AE
:1002F000070707070707070707070707070707078E
:10030000070707070707070707070707070707077D
:10031000070707070707070707070707070707076D
:10032000070707070707070707070707070707075D
:10033000080808080808080808080808080808083D
:10034000080808080808080808080808080808082D
:10035000080808080808080808080808080808081D
:10036000080808080808080808080808080808080D
:1003700008080808080808080808080808080808FD
:1003800008080808080808080808080808080808ED
:1003900008080808080808080808080808080808DD
:1003A00008080808080808080808080808080808CD
:1003B000546D725100000000546D7220537663003A
:1003C000286E756C6C2900004572726F7220696E20
:1003D00020416C74426C636B51207461736B7320A9
:1003E0000D0A00006D69616F750A00006D69616F2B
:1003F00075320A0068756E6772790A004368656332
:100400006B54696D6572000051436F6E7342310029
:100410005150726F644232005150726F6442330027
:1004200051436F6E734234005150726F6442350015
:0804300051436F6E7342360068
:100438001000000000000000017A5200017C010158
:100448001B0D020010000000180000001875FEFFC8
:100458005804000000000000100000002C000000FC
:100468005C79FEFF3404000000000000100000006A
:10047800400000007C7DFEFF10040000000000002A
:08051000FC8F01000400000053
:040000058000004037
:00000001FF
